:020000041100E9
:10300000002373B52B4D2C4C28006361022601F080
:1030100067F94021FE2221742800284B009601F018
:10302000B1F9002836D1217CFF222800244B0096DC
:1030300001F0A8F900282DD1224BA2899A4226D16D
:10304000E389214A93420DD1204B6361204B2268D2
:10305000002A03D1002B01D043CB43C4280001F048
:103060007DF973BD1B4A934201D00023EFE71A4B51
:103070001A4A1B68934206D9C02304222800217CE7
:103080009B0001F0F5F9114B6361154BDFE700235D
:103090002374EAE7CC233821AC2228009B01217459
:1030A00001F0E6F90028F2D10E4B63610E4BE3818B
:1030B0000E4BCCE7743CFF1F185CFF1F245CFF1F06
:1030C000265CFF1F59590000830500000D410011C7
:1030D00068BC0011821500003C5CFF1F87130000D4
:1030E00074BC0011C5410011AAAAFFFF5CBC00110D
:1030F000F7B5164B0192C318021D002000938823D8
:103100005B05D3181B685C1C1AD09CB2402C18D8E5
:103110008D781E0CAC466746CD782D023D43AE42FD
:1031200006D1019800280ED110000C70240A4C70B2
:1031300003249BB20733A343D218009B9A42DED3E9
:10314000FEBD4432F9E71000FAE7C046FC0F00006C
:10315000802213B503000324019189B25201073183
:103160009B18A14304305A1A88235B05C3181B68B7
:10317000591C03D190429241104016BD99B240298A
:1031800007D80B000733A343C0189042ECD30020AC
:10319000F3E74430F9E7134B134A1B68126810B584
:1031A000FA24934201D81A00F824104BE4021B6859
:1031B0009A4210D813000E4A12689A420ED3013375
:1031C00007D1F823DB029C4203D10A49054808F0E5
:1031D0008FFB200010BDFC24E402ECE7FE24E40297
:1031E000F7E7C04600C0071100D0071100E0071143
:1031F00000F00711FFFFFF7FF0B59BB015000490B2
:103200000391402A00D9A0E006AB59801A80FFF74D
:10321000C2FF0400042816D9002206A9FFF768FFA0
:10322000052810D906AB1B88AB420CD1002D07D066
:10323000514B2A000499C01808F0B2FA002802D1B4
:1032400001201BB0F0BD06AB1D8020000699FFF7E2
:103250007FFF041E7BD1069B0793FFF79CFF802313
:103260005B01C618802307001B039E4201D3F8268A
:10327000F60288235B05F31801931B68013302D023
:10328000019808F0ADFB3D49019808F031FB3B1D6A
:103290000293331D05938822029B52059B181B68DD
:1032A00008935A1C3CD044219AB20091402A04D879
:1032B0000320D11D814389B2009103991B0C8B42DD
:1032C00024D0402A22D80122300008A9FFF710FF9D
:1032D000021E1BD1380008A9FFF70AFF04000428CA
:1032E00031D9009A059B9B1880225201B218934253
:1032F00040D288235B05C118009A09A808F030FA6B
:103300001D4B009A09A9F01808F072FB009A029B65
:103310009446634402931A4B029AFB189A42BAD31A
:1033200088235B05FC1821680198013908F0E0FA50
:10333000200008F055FB039A07AB5A80300007992C
:10334000FFF706FF0400002C03D1002079E70428D2
:10335000FBD988235B05E018069908F0C9FA032316
:10336000EA1C9A4300D16BE7034B0499E01808F07C
:103370003FFB65E70424ECE704000011FFFFFF7F3B
:10338000F80F0000F7B505001400402A21D80027E7
:1033900001AE71803780FFF7FEFE042816D93A008F
:1033A0003100FFF7A5FE042810D93688BC420BD0A7
:1033B000BD4209D0221CB44200D9321C064B92B245
:1033C000C118280008F0CCF930B2FEBDC04300B2ED
:1033D000FBE703204042F8E70400001137B5042260
:1033E00004000D0001A81649FFF7CCFF02000428D5
:1033F0000BD1019BA34208D3AB4204D0104901A8D2
:103400000195FFF7F9FE01203EBD0E4C2368200018
:10341000019308F0E5FA019920000139019108F0C3
:1034200067FA80235B01E418074B9C42EED104222B
:10343000034901A80195FFF7DFFE0020E4E7C0463D
:103440005555000000C007110000081130B589B0C3
:1034500008F0EEF810226946254808F061F9254B7E
:10346000009A9A420ED1019B029A0F2B33D8002169
:1034700001240698013B08D2002900D00292029B49
:10348000013331D10023029325E0551CF2D1020013
:103490002100EFE710341022200004A908F040F9C1
:1034A000029B013301D1069B0293882304995B059B
:1034B000C918059B06981A03120B049105928142C4
:1034C00003D02B4201D108F04BF9019B013B019342
:1034D000019B002BDED1029B002B03D004930498A8
:1034E0004168084709B030BDE025014C2D03EFE7E6
:1034F00000000111504859368022F8B5964C974B80
:10350000D200002120001C6008F052FA2300944AE7
:1035100088331A60934B1A786A23002A00D011333B
:10352000E3620A232365904B37221B780821A363AB
:103530008E4B6018E361102323628D4B3B25636142
:10354000C823DB00A36123008C331A602823013ACF
:10355000E26321646364C267043A201DC2672000ED
:10356000BC3005602000C03001602000C430036022
:1035700020000635CC3005602000083DC8300560CD
:103580002000D03002602200D43211602200D832F4
:10359000136022000226E032200016604222DC3056
:1035A000026020001B3DE43005602000E83001602F
:1035B0002000EC30036023000520F4331860230062
:1035C000F0331A602300183290331A6023009433CA
:1035D000196023001E3A98331A60AF23DB00236082
:1035E000644BFA252363644B6448A3642300B93217
:1035F000FC33FF32AD00A260E56022611D60A06275
:103600007320E0656D386065A065FA2796203F015C
:103610008000E76465625960A0660920E0660020CA
:10362000616757496666E167564E57492667A06746
:103630000F601527676027001A219C373960270023
:103640000731A037396027004B49A837396021007E
:10365000F8310D6021006427A4310F6021005F3F25
:10366000AC310F602100033FB0310F602700B43749
:103670003D00C8272F6027003825B83738609D6087
:10368000424D96215D64424D8900DD61414D1962D4
:103690005D62F53DFF3D9D621E253949DD66596637
:1036A000996499673C49DE651E6618675867D96753
:1036B000BE233A495B00E1508130394BFF30235043
:1036C00004302150C42149006350C623E4205B002C
:1036D000E2500433E2503349334A344BD160344929
:1036E000800019503349E938FF3819503249043005
:1036F000195032493248D16132491163324951631C
:103700001900F4310860CE20304940001160304982
:10371000195019002F48F83108602F49D1658221CE
:103720002E4A89005A501A002D490832D1671A00D2
:103730002C49B432116088212B4A89005A501A0052
:103740002A49883211602A4ADA6408F0D9F901203E
:1037500008F0AEF8F8BDC0460004FF1FC45EFF1FAE
:10376000A069FF1FAC3EFF1F4A0AFF1F3A07000077
:1037700080C3C9019A02000050C300006A1800000B
:1037800088130000204E0000F009FF1F6509FF1F8D
:1037900068100000C4090000DC05000040420F0072
:1037A00010270000D91AFF1FFC00FF1F0000FF1F99
:1037B0009527FF1FD92AFF1F7129FF1F251EFF1FF5
:1037C0007523FF1F411EFF1FED1FFF1FB11DFF1FB0
:1037D0000124FF1FE924FF1FD918FF1FB923FF1F72
:1037E000C921FF1FD521FF1FB11CFF1F691DFF1F2E
:1037F0009D1CFF1F0223F0B501245D4D5D4E2B7013
:103800005D4B91B01C705D4F039333680021200025
:10381000BB7006F0B9FD200006F0B0FC0023984212
:1038200005D0BA78552A02D0332A00D094E033600C
:1038300007F07EFEFFF760FE1F2201240021504B9F
:1038400036261A704F4B1C704F4B19704F4B19682E
:103850009143163A0A431A60602219689143403A2C
:103860000A431A6008F03CF807F092FEC120FF21DD
:10387000474B80001A588A431A50C5229200985824
:103880008843BF39014399509858424908408021E4
:10389000C9010143802099509958C0050902090ABD
:1038A0000143995080213C48490108F031F9032334
:1038B0002200009339490194394807F049FF2E222C
:1038C000384904A807F04CFF02AB04ACF618617845
:1038D0002078023406F072FCA642F8D1324C334B09
:1038E000226803201A40A023DB02134323608023B5
:1038F00022689B041343236022682D4B1A408023C7
:103900009B03134323602B4A2B4B934200D8012087
:1039100008F05EF807F0FCFE80232268DB04134306
:103920002360287808F014F9039B1878C0B207F0D8
:10393000A7FE07F0CDFE2149042007F021FF06F085
:1039400057FE00F0A9F800F0E9FD00F07BFE00F062
:103950000BFA002011B0F0BD00932100174A04209B
:1039600008F066F88023DB059C62FFF76FFD5FE7D8
:103970004A0AFF1F34F00040AC3EFF1F485CFF1FA7
:10398000480AFF1F490AFF1F680AFF1FBCF00040DA
:1039900000E100E0FF00FFFFB03EFF1F3451FF1FBA
:1039A000B04EFF1F80BB001114F00040FF7FF8FFF6
:1039B000FFFF9FFF0080FF1FA069FF1F3B00010862
:1039C00070B500252549264A26484D6308CA1B05BF
:1039D0001B0DED188242F9D100268022224B920560
:1039E0008B630921214B224C1E62224B1120DA6786
:1039F000214BDA688A43DA609A6820490A409A6063
:103A0000266007F07DFF112008F062F8636C1C4A05
:103A100013406364EE24E4006C431A4A200C040053
:103A2000642390420AD8FA223300D200904205D98A
:103A3000154B0A21C01808F00BF8C3B2134A112025
:103A40001372D48007F07CFF114B1B78002B04D13C
:103A5000104B1021187807F013FF70BD00000540CF
:103A60000806054080060540FF01000000F0004008
:103A70000038004004E100E03CF00040FFDFFFFFC1
:103A8000FFFEFFFFB70B000030F8FFFF305CFF1FA9
:103A90006A5EFF1F685CFF1F002210B51100112035
:103AA00007F02EFE10BD0000F8B500230926364FA2
:103AB000364C3B62E3681120B343E36008F008F83A
:103AC000112007F01DFF112007F03AFD4023226866
:103AD00010251343236080236268DB021343636075
:103AE0008023A26802211343A360A368284A082008
:103AF0001340A3608023A2689B0113430122A360AB
:103B0000236CAB432364236C1343236480231B0186
:103B10003B62226B1F4B1A402263626B1A40626346
:103B2000A26B1A40A263E26B1340E363E3681A4A94
:103B30001340E36006F042FB0121082006F052FC2E
:103B40008023164A5B00516C11200B43536407F02D
:103B500037FDFD21C720124B124A89005A50A36B32
:103B600080002B43A363E3680F4A3343E3600F4BAA
:103B700019581140802212020A431A5080229205DD
:103B80001A600B4B5D63F8BD00F000403CF0004054
:103B9000FFFFDFFFEFFFEFFFFFFF7FFF0038004079
:103BA0000000FF1FC1390011FF00FFFF00E100E02E
:103BB0000000054030B503A804880B20002C0ED16E
:103BC0004968074D08784978090201430A20A9424B
:103BD00005D1012120001980024B1B7A137030BDE2
:103BE000192A0000305CFF1FF7B5150008AA1688D7
:103BF0004A680F4F14785278120222430A24BA42BC
:103C000014D10122DBB2019200962A0007F02AFCAF
:103C1000041E0BD1074B1B68002B07D068782A784D
:103C20000002104342425041013098472000FEBD3F
:103C300002290000B45BFF1F30B5012503790400A1
:103C4000BFB02B4211D00A49408806F077FF2842C6
:103C50000BD0084B01A95B8D4D800B80064B0022D9
:103C60001B7A60880B7104F071F83FB030BDC0461C
:103C7000AC5BFF1FE83AFF1F305CFF1F10B5054922
:103C8000054806F011FF0421044A054806F0CEFE5F
:103C900010BDC046AC5BFF1FFFFF0000B0BB0011B2
:103CA000E83AFF1F10B5024804F0D2FE10BDC0462E
:103CB000393C0011062310B5837010330371443B67
:103CC00043712A3383714433C371002302220121DB
:103CD00003720E4B027041701C8881724472197A13
:103CE0000273C1729A784273DA7882730322C273C4
:103CF0001A7902745A7942740C2282749A79C274C5
:103D0000DB7903751123C370152010BD305CFF1FD4
:103D100010B5142007F00CFD124B1422002118607E
:103D200007F046FE002007F023FF012007F060FCAB
:103D3000022007F0C5FD032004F02EF9042006F050
:103D400043F9052003F06CFB062004F039F8072046
:103D500001F036FA082006F049FE092001F01EF8AD
:103D600010BDC046B85BFF1F07F04AFC012007F0FA
:103D70006FFC07F08DFE0000094B10B5040098425F
:103D800005D0012904D12000064906F08DFE10BDA2
:103D90000229FCD1013904F019FE0028F3D0F6E71E
:103DA000FEFF0000DE5BFF1F70B50D7A100004AA55
:103DB0002C00168810221440154220D1002E20D14C
:103DC0000A78022A18D14A68517815780E4A0902F1
:103DD0002943914205D00D4A914209D01C800A2402
:103DE00004E014220A491A8007F0BAFC200070BDD2
:103DF0000C2208491A80F7E71C800124F6E7082402
:103E0000F4E70B24F2E7C046F3FF0000F4FF0000E4
:103E10003C3DFF1F8CBC001110B504000749084849
:103E200006F042FE074804F053FD0020E40704D5E5
:103E30000721054A054806F0F9FD10BDDE5BFF1FAE
:103E4000FFFF0000793D0011F4BB00112C3BFF1F68
:103E500000B50C4BBFB01A780B4902A800F0ACFCBF
:103E60006B4680B2D880002809D06A46074B01A96A
:103E70001B889380064B0022188803F067FF3FB031
:103E800000BDC046BC5BFF1FBD5BFF1F863BFF1F25
:103E9000903CFF1F00B50C4BBFB01A780B4902A82D
:103EA00001F09AFE6B4680B2D880002809D06A469D
:103EB000074B01A95B8D9380064B0022188803F005
:103EC00045FF3FB000BDC046E65BFF1FE75BFF1F3D
:103ED0002C3BFF1F903CFF1FF7B50E00377A1C00EC
:103EE00008AB11003D001A8820231D401F423CD121
:103EF0003378022B3BD173681F785B781B023B43FE
:103F00001E4FBB4208D01E4FBB4214D01D4DAB42CA
:103F100021D00A252800FEBD002A2AD1142C2AD837
:103F20002200F06807F01CFC174B1C70012CF1D923
:103F3000FFF7B0FFEEE7002A1BD1202C1BD8220090
:103F4000F06807F00DFC114B04211C70104B187821
:103F500007F096FCDEE7E3B20124009201940A0028
:103F6000310007F07FFA0500D4E70825D2E70125E4
:103F7000D0E70B25CEE70D25CCE7C046F3FF0000C8
:103F8000F4FF000002290000E65BFF1FBC5BFF1F7F
:103F9000685CFF1F332310B5040003700A22074931
:103FA000013007F0DDFB064B0F201B681A0AE37295
:103FB00022731A0C1B0E6273A37310BD305CFF1FBB
:103FC000585CFF1F30B5012503790400BFB02B42B8
:103FD00013D00B49408806F0B1FD28420DD06A4647
:103FE000084B02A81B889380FFF7D4FF6B46D8804C
:103FF0000022608801A903F0A9FE3FB030BDC04691
:10400000DE5BFF1F863BFF1F10B5024804F020FD5A
:1040100010BDC046C53F001170B5160004AA148833
:1040200005AA15784A685078117800022A4A084390
:10403000801805284BD807F02BFB03131E29343FAB
:104040000720032C0BD80422121BAA4200D92A00F5
:1040500022491A803000091907F082FB002070BD48
:104060000720112CFBD81222121BAA4200D92A00C9
:104070001B491A80EEE707200E2CF0D80F22121BE6
:10408000AA4200D92A0017491A80E3E70720032C27
:10409000E5D80422121BAA4200D92A0012491A802C
:1040A000D8E70720032CDAD80422121BAA4200D931
:1040B0002A000E491A80CDE70720032CCFD804220E
:1040C000121BAA4200D92A0009491A80C2E700221D
:1040D0000A201A80C3E7C046DCD5FFFF3FBC0011B1
:1040E000045CFF1F2FBC00112ABC001125BC00116D
:1040F00020BC001110B50D21024A034806F096FCC1
:1041000010BDC04614BC00119C3BFF1FF0B500243D
:10411000274E85B03000B47100F0E2F8254D264BF3
:10412000EA89297C9A422FD10423300003AA00F0A7
:1041300057F90400300000F011F90123B371002C8D
:1041400034D16B4699892B68C9BA4B4329891B4ADC
:104150001B145B1853806B46D9896B6849BA89B2C6
:104160004B4369891B0C5B181548191C1BB2834211
:1041700000DD011C0B0400D5002113889180013360
:104180001380200005B0F0BD0227220003AB3000F1
:10419000009700F0F7F80E230400297C012230007C
:1041A00000976B4400F0EEF80443C3E71C00E8E717
:1041B000743CFF1F185CFF1F83050000305CFF1F6D
:1041C0000F27000073B5234E300000F089F8224D10
:1041D00007236A463000297C00F002F90400300011
:1041E000002C33D16B461B787F2B2FD800F0B6F80C
:1041F0006B46D878F02302041B031A406B469B8859
:1042000016495BBA9BB21A432B68000953432A89AB
:104210001B0C9B184B806B465A789B7812031B0132
:104220001A436B68024353436A891B0C9B180C4862
:104230001A1C1BB2834200DD021C130400D50022AD
:104240000B888A8001330B80200076BD00F086F851
:104250000124F9E7743CFF1F185CFF1F305CFF1F4F
:104260000F27000070B5114C237C002B0FD0382B8A
:104270000ED10F4D280000F033F8CC23AC222800DB
:10428000217C9B0100F0F4F8280000F067F870BD75
:10429000084BE2899A42FAD1054D280000F020F837
:1042A00000222800217C00F0C5F8EDE7185CFF1F14
:1042B000743CFF1F8305000010B5084B1A7C002AD0
:1042C00009D05B69002B06D09847041E01D0FEF789
:1042D00097FE200010BD0124F9E7C046185CFF1FBF
:1042E00070B5C17905000C00631E9C411A4BE402B5
:1042F000E41849000460C9B2007906F0A9F8E97928
:10430000687949000131C9B206F0A2F8E8790930AC
:10431000C0B207F015F90023E36661332360AA7980
:104320005B3B002A0ED022689A43023B1343236072
:104330000A23E3610733236200232363A36301336A
:10434000E36370BD22689A4302231343236046232C
:1043500063610633A361EFE70050004070B50025AC
:1043600004000368DD66C0790930C0B207F0B0FB15
:104370002900207906F008F82900607906F004F891
:1043800070BD0000F8B51E0006AB1D780023046860
:104390001700E366616007F04BF901238022E366B2
:1043A0002B0027615200013B08D207F031FA0820A8
:1043B0000A4A1168002D03D12800F8BD2261F2E7F6
:1043C000236F034203D02369013D33700136136824
:1043D0005B1A032BEED90125EEE7C0466008FF1FEC
:1043E00070B51C00002305681600EB66696007F0D5
:1043F0001FF901238022EB6623005200013B08D203
:1044000007F006FA08200A4A1168002C03D12000A0
:1044100070BD2A61F2E72B6F034203D02B69013C88
:104420003370013613685B1A032BEED90124EEE7D3
:104430006008FF1F002370B504681500E366616023
:1044400007F0F6F80123E366256107F0E1F9802023
:10445000064A80001168636B034205D113685B1A3A
:10446000032BF8D9012070BD0020FCE76008FF1F76
:1044700070B51D00002304681600E366616007F054
:10448000D7F80123E36626610F33626B1A42FCD032
:104490002B0A23611023626B1A42FCD0EDB2256116
:1044A00007F0B6F98020074A80001168636B034269
:1044B00005D113685B1A032BF8D9012070BD0020C9
:1044C000FCE7C0466008FF1F70B51E0000230568AA
:1044D0001400EB66696007F0ABF80123A619EB66E0
:1044E0000F33B4420ED107F093F980200A4A8000BE
:1044F00011686B6B03420CD113685B1A032BF8D95C
:10450000012070BD21782961696B1942FCD001340A
:10451000E7E70020F5E7C0466008FF1F10B5084C2C
:10452000E368002B08D1074B1B685B045B0C0A3364
:104530006360054B1B68236007F0A2FAA06010BD02
:10454000585CFF1FC8F00040CCF0004010B507F0E9
:104550006FF80F4B996A9A6A8A42FBD10D4C6268D8
:10456000A0688A18121A531E884200D31300A16053
:104570002168DA0B52185B0407495B0C6360226008
:104580000B60064B1A6007F043F9206810BDC04667
:1045900000F00040585CFF1FC8F00040CCF0004025
:1045A00070B51F4C23793F2B01D93F2323711D4B3D
:1045B00022791A701878C0B207F02AF818231A491D
:1045C0001A4A0B801A4913800B805380A37919492A
:1045D00080200B800C21938001334B43164D191C16
:1045E0000001834200D9011C2980D1806379002B0E
:1045F00011D101336371237A012B01D80223237275
:104600006279237A0D4853430A21584307F020FA70
:104610000B4D286070BDA02BEDD9A023EAE7C04662
:104620004C5CFF1F480AFF1F8E3CFF1F583EFF1FB8
:104630008C3CFF1F8A3CFF1F883CFF1F710200005B
:104640003C5CFF1FF8B514210020FEF7C7FE114C9B
:10465000011E114D09D10C22104BC1CBC1C4280041
:1046600007F0A6F9FFF79CFFF8BD0C2220000C49CB
:10467000FEF788FE0C2802D0084B43CB43C40C2223
:1046800028000849FEF77EFE0C28EBD00C22002102
:10469000E5E7C0464C5CFF1F185CFF1F80BC0011A3
:1046A000FC0C0000F50C0000F0B51D4C8022A54468
:1046B0000400882069465201400506F071FF9022EF
:1046C00012016A441300200032C832C316C816C350
:1046D0008023144C144FA6689B033343A3603B60B4
:1046E00006F07EFF8823A0685B05C01807F078F904
:1046F0000025882329008022A0685B05C018401986
:104700006944520007F074F980230135FF355B01DD
:104710009D42EED1A6603E60044B9D44F0BDC04674
:10472000FCEFFFFFCC3DFF1F9808FF1F04100000A7
:10473000F0B5040087B0002825D0684607F080F95E
:104740001B4C022806D106226946200007F028F8F3
:10475000002816D06946002301250F262F00E25CB1
:10476000013310091030874038002F003240974045
:104770003A0002434A610439062BEFD16846FFF73D
:1047800093FF07B0F0BD182269460A4806F008FFFB
:104790006A46A300D358013305D01822FF2168468A
:1047A00007F006F9EAE70134062CF1D1E9E7C04643
:1047B0006509FF1F00090011F0B5002504000E0077
:1047C00085B0AA4200D186E04B1C087801934B7853
:1047D0008978377909021943F3783F061B040B43A4
:1047E0001F43039720706570252800D196E033D8C9
:1047F000112813D807F09CF869002501250125012F
:104800002501AA00B800B1002501250125012501D7
:104810002501250125012501FF001F01232800D1C5
:10482000D8E0DB2800D02EE1042A00D8ACE0102527
:10483000052A05D0551F2A003800711D06F090FF8B
:1048400005223100200006F08BFF2A003900601D90
:1048500006F086FF05353EE0562859D010D833289B
:1048600000D19DE0552839D02628DAD19C4B29006B
:10487000132218001D0007F09BF8FEF7C1FB5CE057
:10488000712800D177E0722800D180E0602800D143
:104890008BE0DC28C5D1022A00D875E07378BFB25E
:1048A0006370B378A370032A05D0033A390092B23B
:1048B000F01CFEF7A1FC10223900E01CFEF762FD9F
:1048C000C51C002807DA60705CE00C2220008549D6
:1048D00006F046FF0C25280005B0F0BD013A824DD8
:1048E0000C2A13D8002A0AD02800019906F038FFB4
:1048F000FFF756FE0C2228007C49FEF77DFC2900BC
:104900000C22601C06F02CFF0D25E4E70C22EBE7DF
:10491000754D774B2A0043CB43C2E9E7013A704D0E
:104920000C2A11D8002A08D00199280006F018FF97
:104930000C2228006F49FEF75FFC29001322601C3F
:1049400006F00EFF1425C6E70C22EDE705226A49A2
:10495000601C06F005FF0625BDE712226749601CB2
:1049600006F0FEFE1325B6E708226549601C06F036
:10497000F7FE0925AFE77178F02905D8614B188853
:1049800001F086FD0225A6E7FF236370FAE75E4B80
:10499000012A03D072785A706270F3E75B78F4E70B
:1049A0002000FFF7F7FA050095E7013A574D072A6F
:1049B0000ED8002A05D00199280006F0D1FE01F09A
:1049C00045F829000722601C06F0CAFE082582E788
:1049D0000722F0E7042A04D94D4D2F6007F050F864
:1049E000A860FFF7B3FD0422039003A9601C06F042
:1049F000B7FE05256FE7474D062A15D90622280080
:104A0000019906F0CDFE00280ED00622019928005B
:104A100006F0A6FE062240492800FEF7EDFB012322
:104A2000394A51780B43537029000622601C06F066
:104A300097FE07254FE7012AA6D07078FFF778FE8A
:104A4000A0E7012800D0ECE6931E344F1A2B04D8BF
:104A50007378002B09D100F015F9314B39001D781E
:104A6000601C6A1E06F07CFE35E7551E2A0001997F
:104A7000380006F075FE2B49AAB23800FEF7BCFBE1
:104A800000F036F9E9E7DA281DD1042A00D87BE7DF
:104A9000082A15D9B37972791B021343F2791204EB
:104AA0001A43337A1B0613433B603B6805223100EF
:104AB0002000039306F054FE0422601D03A956E76C
:104AC000FE236370F1E7DE2800D05DE7511E012A66
:104AD00001D10025FFE6019800F09EFFF9E7C046EE
:104AE000185CFF1F8CBC00114C5CFF1FFC0C00000D
:104AF00080BC0011F50C0000245CFF1F045CFF1F4C
:104B0000D03DFF1F903CFF1F485CFF1F2D3DFF1F46
:104B1000585CFF1F6509FF1FADAC0000495EFF1F19
:104B2000475EFF1FAEDE000070477047020010B501
:104B3000094B0A32094C92B2DA815A829881188262
:104B4000207802F00BFB0422054B012120781A701B
:104B500006F096FE10BDC0465A3DFF1F925EFF1F35
:104B6000915EFF1F013870B5042809D806F090FD4A
:104B7000030928081200234B0221187806F080FE52
:104B800070BD204B0821187806F02AFE00221E4B2B
:104B90001A72F5E7802200241B4B1A4D52001A812D
:104BA00008211A682878DC7206F0CAFF21002878EC
:104BB00006F05EFF012000F04FFE00F047FFDFE748
:104BC000104B0821187806F00BFE1048FFF772F81A
:104BD0000F4B104A9B79002093800F4A138080224C
:104BE000094B5200D8721A8100F036FE00F02EFFF9
:104BF0000A4B5B78002BC3D0094A136006F0C8FD4E
:104C0000BEE7C046685CFF1F3C5CFF1F993CFF1F6E
:104C10004C5CFF1F583EFF1F8A3CFF1F485CFF1F74
:104C200034F0004010B501290BD1012809D1054B02
:104C30001B78002B05D02622034B04485A72FFF73D
:104C400075FF10BD6A5EFF1F3C5CFF1FC4090000BA
:104C50000300F0B50A4D8E18B14202D152008018FF
:104C6000F0BD0C782F6824093C5D0F271C700C7870
:104C700001313C402F683C5D5C700233ECE7C0467C
:104C8000843CFF1F0D22114B10B51A700C23104CE1
:104C900010492370093A033B0F48637006F060FD2A
:104CA0002D2301220D490E48A371FFF7D1FF0122E8
:104CB0000C49FFF7CDFF01220B49FFF7C9FF002286
:104CC0000A491000FEF798FA10BDC046665EFF1F45
:104CD000475EFF1F3FBC0011495EFF1F6709FF1FB2
:104CE0004E5EFF1F6609FF1F6509FF1FAEDE000055
:104CF00070B5124C132220001149FEF743FB114DF1
:104D0000002817DDAB78002B14D0431C2B7009232F
:104D10006B70002300190370287829000130C0B29D
:104D200006F08EFC297822000139C9B2002005F076
:104D30009BFD70BDFFF7A6FFEEE7C046495EFF1F73
:104D4000AEDE0000475EFF1F10B5114B1A781870D9
:104D5000002A0ED000280BD10E4B1A78062A07D84D
:104D60005423D340DB0703D50B4B187802F0F6F938
:104D700010BD0028FCD0074B1B78012B02D0033B51
:104D8000022BF5D8044B0121187806F079FDEFE7E6
:104D90006A5EFF1F915EFF1F925EFF1F70B54A4E55
:104DA0004A4A4B493070012005F000FC00F0B2FE89
:104DB000FEF726F906F0E4FD032246494648FFF7D0
:104DC00047FF2D24030004221C7044490130FFF7E3
:104DD0003FFF30230470424D424C437083702E3BA2
:104DE000062220004049EB87FEF7CCFA062813D0B4
:104DF000200006F025FE022809D00321200006F03D
:104E00002FFC8D23E3706E3B2371193363710622EF
:104E100020003549FEF7F0F9344B1B68FC335C6425
:104E2000FFF766FF0020FFF78FFF314C314A012169
:104E3000314B1278207802F053F9304A304B127817
:104E40000021207802F04CF901222E4B1A702E4BD3
:104E50009B78552B31D12D4B3B325A722C4B2D4A1E
:104E6000AB81EA812B826A822021307806F020FC17
:104E70000120404205F044FD0120404205F0E0FDE4
:104E8000FFF738F9FEF7FAFE00F0A4FC01204042DB
:104E9000FEF7C2FF012006F063FBF02001F0DCFA10
:104EA0000121307806F0ECFC307802F0B3FA1A48B1
:104EB00006F0B6FCFEF7F8FD70BD6422174B5B7977
:104EC00053431A000A32CBE7685CFF1F294B0011DD
:104ED000254C0011D03DFF1F045CFF1F245CFF1F09
:104EE0005A3DFF1F6509FF1FADAC0000C45EFF1FE8
:104EF000925EFF1FB83CFF1F993CFF1F665EFF1FBD
:104F0000475EFF1F385EFF1F485CFF1F3C5CFF1FB2
:104F1000C4090000CE0900006A5CFF1F4C5CFF1F43
:104F2000F8B50A0020230D001A40194257D0574BFC
:104F30001B78002B50D0FFF709FB554B554C564EB4
:104F400099686268737A8A1ADB039A4202D36160B5
:104F5000FEF7AAFD327A217A531EDBB2994205D1BF
:104F6000FFF780F9002000F0A7FD0FE09142F9D390
:104F700000232372FFF7A0F9012000F09DFD474FA9
:104F80003800FEF797FE390006F03AFD637A002BF1
:104F90001FD0013BDBB26372002B1AD1404B9B78D0
:104FA000552B01D106F0F4FBE37A002B0CD0002343
:104FB0003C4A3A4FE3721388380001331380FEF7FE
:104FC00079FE390006F01CFD642370795843FFF721
:104FD000ADFD237A0133237220206840F8BD0BB267
:104FE000002B0ADA304B187806F082FD002801D039
:104FF00006F0A6FB80200002EFE70224214206D043
:10500000244B01201A72FFF79FFE2000E5E70B07F3
:105010001ED5FFF79BFA1E4B1E491F4C98684A6825
:10502000637A821ADB039A4202D34860FEF73CFDA2
:10503000FFF742F9FFF716F9012000F03DFD00F0FF
:10504000E3FB2368DB0701D5FEF7DEFF0820C4E79A
:105050001024214206D00D4B1B78002BD5D1FEF732
:1050600021FED2E70124214207D0104800F06CF85D
:1050700006F0F6FB00F006FDC7E704240800204018
:105080002142ABD0FEF7E4FEBFE7C0466A5EFF1FD9
:10509000585CFF1F3C5CFF1F4C5CFF1F993CFF1FCF
:1050A000485CFF1F305CFF1F685CFF1F7C3CFF1FDC
:1050B000F0B51B4B1B4F1B883A8804001A4E1B4D42
:1050C00085B09A420DD832889A420AD3184B1A8872
:1050D0002B889A4205D1174A174B12881B889A428F
:1050E0001BD0052001F00EFA3B8802AA13803388FA
:1050F000019053802B88114D93800F4B02A91B8880
:10510000D3800F4B2A78188802F02AFF0D4B082114
:105110002878019A1C7006F003FD05B0F0BDC0466A
:10512000365EFF1F8E3CFF1F8C3CFF1F8A3CFF1F1B
:10513000345EFF1F325EFF1F883CFF1F925EFF1F21
:10514000903CFF1F305EFF1F13B50C4B1C78002CEA
:1051500011D1002801D00A4B18600A4A0A4B117875
:105160000A4A10780A4A01920A4A0092002205F07F
:1051700073FA200016BD1124FBE7C046915EFF1FA5
:105180002C5EFF1F905EFF1F805EFF1F925EFF1F61
:105190006C5EFF1F705EFF1F10B5064B12201B7860
:1051A000052B06D1044B13221988044B187801F003
:1051B00085FB10BD915EFF1F903CFF1F925EFF1F9D
:1051C00010B500240122114B52421870104B1C7074
:1051D000104B1A8002F01EF904220F4B21001A70A6
:1051E0000E480C3206F024FB102221000C4806F079
:1051F0001FFB07220B4B1C600B4B1C700B4B1C70D6
:105200000B4B1A700B4B1C7010BDC046925EFF1FFB
:10521000915EFF1F903CFF1F905EFF1F805EFF1F8F
:10522000705EFF1F6C5EFF1F465EFF1F455EFF1F27
:10523000923CFF1F445EFF1FF8B5174C060025780F
:1052400006A814240078052D23D1B41F134FA5B24E
:105250001824BD421DD88D1FADB2BD4219D8FA2504
:105260006D00AA4215D21D000D4F0A3DADB2BD42E0
:105270000FD80C4C26800C4C21800C4900240A804D
:105280000B4A1380FFF714FF0A4B0421187806F02D
:10529000A7FA2000F8BDC046915EFF1F790C000000
:1052A000750C00008E3CFF1F8C3CFF1F8A3CFF1FCB
:1052B000883CFF1F925EFF1FF0B50BB20D0089B056
:1052C000002B00DB70E1A44E307806F011FC041EC8
:1052D00050D00378A22B00D122E1D02B1AD0912BF1
:1052E00045D143780E2B42D19C4B82889A423ED1C5
:1052F0009B4A83681278052A39D1032018567F28E3
:1053000035D0984B1B68002B31D05B68002B2ED01A
:1053100098472CE08078072829D806F0B9F90428A6
:10532000183F3F74A8D86378002B0CD101218C4B17
:1053300019708D4B1A78002A5BD08C4B307801F0B5
:10534000CFFE002855D00722854B1A7051E06178B6
:105350000029F8D1E378002B11D0854A854B1278CB
:10536000307801F0BDFE60706378002BEBD1200037
:1053700006F0E6F980200002684009B0F0BD784BE5
:105380001B78022BF3D00121307806F089FA00282F
:10539000EAD10121307806F073FAE5E76378002B53
:1053A000D1D16F4F032807D13B78052B02D10133B0
:1053B0003B701EE00223FBE76F4B1A886F4B029392
:1053C000002A0BD01B78002B03D00121307806F087
:1053D000A7FB3B78062B04D1013BE9E7029B1A703F
:1053E000F7E7042B41D10121029B3078197006F0B8
:1053F00047FA5C4B1B68002BB9D01B68002BB6D05A
:10540000574A107884E76378554F002B27D106223E
:10541000211D5B4806F0A4F962895A4B5A491A804B
:10542000A2895A4B1A80E3890B80052139705849AB
:105430000A80584A1380228A574B1A80574B1B7890
:10544000012B09D11F2001F05DF8FA22920042439E
:105450000421307806F064FB0022484B75E7312BBD
:1054600000D070E70022454B1A700323A0E7062204
:105470000021434806F0DCF90023454A042113804B
:10548000444A30781380444A138006F0A9F9082171
:10549000307806F0A5F9A379083B5A425341304AC7
:1054A00003331370304B1B78002B06D0334B30780E
:1054B0001A78002A06D001F051FE0122314B5242E7
:1054C0001A8096E70121197006F0DAF9F5E708214C
:1054D000307806F085F96378002B00D047E72C4B35
:1054E0002D4F0293E388029A04211380294B3078D0
:1054F00003932389039A138063893B8006F0D0F9D4
:10550000002800D033E7264B1B68002B00D12EE784
:10551000039902983A88098800881B68984726E70B
:105520004379132B00D022E70389012B0AD11D4BAD
:105530001B78022B06D10821307806F051F9FFF7CD
:105540002BFE14E7052000F0DDFF08210200307873
:1055500006F0E6FA0BE7C046925EFF1F0514000056
:10556000915EFF1F2C5EFF1FB83CFF1F993CFF1F81
:10557000665EFF1F475EFF1F685EFF1F6A5EFF1FBC
:10558000395EFF1F903CFF1F405EFF1F425EFF1F02
:10559000365EFF1F345EFF1F325EFF1F385EFF1F47
:1055A000285EFF1F305EFF1F8020C001014200D037
:1055B000E2E6CB0731D5324B1B78002B1DD0314EA4
:1055C00005AC3378052B1AD1023B23702E4B2100FA
:1055D0001B7823722D4B1B7863722D4B187801F0CA
:1055E00023FD002809D007202A4B30701B68002BB0
:1055F00003D01B68002B00D098470120BCE60E208A
:10560000254B06221B7825492370254B1B78637098
:1056100002ABC01806F0A4F8D8E70223080018402F
:10562000194209D0174B1B78052B03D11D4B188845
:1056300005F0F6FF02209FE60424214203D0FFF785
:1056400037FD200098E6082308001840194200D1D1
:1056500093E6154B1C78012C03D0022C0DD00820AA
:105660008AE6124B124A134913481B88128809888C
:1056700000880094FFF7E0FDF1E7FFF78DFDEEE70E
:105680006A5EFF1F915EFF1F923CFF1F445EFF1F7B
:10569000925EFF1F2C5EFF1F465EFF1F933CFF1FA5
:1056A000455EFF1F903CFF1F305EFF1F883CFF1FC1
:1056B0008A3CFF1F8C3CFF1F8E3CFF1F10B502A8C9
:1056C00004880B20002C10D1496808784978090219
:1056D00001430C48814209D1022119800A4B5988A3
:1056E0001170DB7800205BB2537010BD074C0A20AC
:1056F000A142FAD102211980034B998811705B797C
:10570000F0E7C0466E2A0000305CFF1F6F2A0000E1
:10571000F7B5150008AA16884A680F4F1478527812
:10572000120222430A24BA4214D10122DBB20192AE
:1057300000962A0005F096FE041E0BD1074B1B684D
:10574000002B07D068782A7800021043424250416B
:10575000013098472000FEBD02290000A45EFF1F13
:1057600030B5012503790400BFB02B4225D0144980
:10577000408805F0E3F928420CD0124B01A95B8D5B
:1057800000220B8002234B800F4B5B888B8060884C
:1057900002F0DCFA0D49608805F0D0F9C0070CD59D
:1057A0000B4B01A91B8800220B8002234B80064B68
:1057B0009B888B80608802F0C9FA3FB030BDC0463C
:1057C0009C5EFF1FBC3CFF1F305CFF1F945EFF1FF1
:1057D000163DFF1F10B5074C0749200005F064F97E
:1057E0002000064905F060F90721054A054805F043
:1057F0001DF910BDFFFF00009C5EFF1F945EFF1FA0
:10580000ACBC0011BC3CFF1F10B5024803F020F9EE
:1058100010BDC046615700110221430888400B406B
:105820000A31084003430E20024AD17881430B43DA
:10583000D37070472D3DFF1F064A1379410705D5E8
:1058400080210B4380011371907170477F210B40C1
:10585000F8E7C0462D3DFF1F054A5378002803D0C6
:1058600080210B43537070477F210B40FAE7C046FD
:105870002D3DFF1F0F21114BDA780A40DA705028B6
:1058800010D901310A43DA702022D9780A43DA703C
:105890004022D9780A43DA708022D97852420A43EA
:1058A000DA7005E03C28EFD82828F1D81428F3D87E
:1058B0000122D9780A43DA707047C0462D3DFF1F98
:1058C000F8B57F23324D04006E789E43314B9842E9
:1058D00005DD76232B70363B33436B70F8BD2E4BC2
:1058E000984203DA58232B701433F5E783B21A0079
:1058F00000215F32294892B2294F297082422DD966
:10590000A9708C4203DA5B421CB220232B70053451
:1059100020B20A2106F09CF804B2FA239B009C42B4
:1059200033DB80232A785B4213432B7064212000F1
:1059300006F08EF80A2100B205F062FF09B22A785B
:105940007B5C13432B700A21200006F081F80A21AA
:1059500000B205F055FF09B27B5C0AE08022AA7014
:10596000002CDADA5B421CB220232B705F23092C57
:10597000E9DC1E430A2120006E7005F041FF09B2E8
:10598000AA787B5C1343AB70A8E7632CCEDCEDE711
:105990002D3DFF1F1B4E00001DFCFFFF2A080000CD
:1059A000D6BC00117F23F7B5194FCD013E79040015
:1059B0009E433E71EDB2632806DD093B33433B71E4
:1059C00040231D437D71F7BD0300093304DA5823DA
:1059D00033433B716C23F4E70E4B019300280BDA41
:1059E0000423444224B23B710A21200005F008FF41
:1059F000019B09B25B5CE4E70928F5DD0A2106F0AA
:105A000027F8019B00B21B5C1E433E71ECE7C046C9
:105A10002D3DFF1FD6BC0011F8B50A4F05003B789D
:105A20000E00002B0CD0084C2000FEF759FC330070
:105A30002A0020003978FEF747FD2000FEF78EFC93
:105A4000F8BDC046B05EFF1F343DFF1F70B50A4E63
:105A50000A4D07223100280005F0A2FE002809D0D7
:105A6000074C31000722280005F07AFE08212000AB
:105A7000FFF7D2FF70BDC0462D3DFF1FA95EFF1F7F
:105A8000A85EFF1F7F2210B50A4B59789143033A55
:105A90001A70103A0A435A7078220E219A70DA78F6
:105AA0008A43DA7006221A7130325A71FFF7CEFF3C
:105AB00010BDC0462D3DFF1F10B5002824D0134C4B
:105AC0000A210223E05E05F0C3FF00B2FFF7F8FEF3
:105AD0000423E05E642105F0BBFF012100B2FFF763
:105AE00061FF207AFFF7C6FE0320FFF795FE002036
:105AF000FFF7A2FE064B1878053843425841C0B262
:105B0000FFF7AAFEFFF7A2FF10BDC046305CFF1FE3
:105B1000915EFF1F70B50024094D2800AC71FEF79F
:105B2000DFFB10233E212800064AFEF7CDFCA042F1
:105B300000D13E34044B28001C70FEF70FFC70BDF2
:105B4000343DFF1FC6BC0011B05EFF1F0200F0B560
:105B500001270A480A4E51188B1A002B00DCF0BDB1
:105B6000082415784308684038404000805B013CB9
:105B700058406D08002CF5D10132EDE7FFFF000021
:105B8000E6BC0011F0B500250F269D4200DBF0BDFC
:105B90004C5D070944403440A400A05801357840CA
:105BA000F3E70000F0B589B06A460D000B000F273F
:105BB000110010351C780133260024093E40167070
:105BC00054700232AB42F5D12023024AFFF7DAFFCC
:105BD00009B0F0BDECBC0011F0B54E780B7889B07F
:105BE00036020C00170001901E43012A61D9954B23
:105BF0009E4200D877E001339E421CD1062A17D17D
:105C0000CA788B7812021A430B791B0413434A7922
:105C100012061A438C4B5A6100221A705A808B4A22
:105C20005A608B4A9A608B4ADA60002009B0F0BD56
:105C300088225205EEE7884B9E423CD182498B7800
:105C4000002B00D0F6E00C2A31D10F22A378934329
:105C5000E278120213432279120413436279120686
:105C600013434B60E279A07912020243207A0004C8
:105C70001043627A12060243CA60E27AA07A1202E4
:105C8000024376484A81834208D804236E4914228D
:105C900001980B7005F064FD1420C7E71201D218BB
:105CA00089235B059A42F0D801238B70BDE7022A55
:105CB000FAD00523EAE76A4A01239642E6D1FFF7C4
:105CC0006BFA052F0CD9E378A2781B0213432279D3
:105CD00012041A4363791B061343624A0393136049
:105CE00005F056FDA1E7584D2B78002B9DD1AB78E0
:105CF000002B00D1A0E02B8901339BB20093B3426B
:105D000000D091E0132AD4D9CF7C8B7C3F021221A2
:105D100020001F43FFF71AFF874200D08EE0002EBD
:105D20003DD1E378A2781B0213432279E96812047B
:105D30001A4363791B06134303930A228B4212D141
:105D4000FF23A370E370237163716B89002B09D16A
:105D5000E37B227C1B0212041343A27B13431B0927
:105D600001336B8100226B89002B8ED0002A67D112
:105D7000686837013818000B6B690003039098427C
:105D800005D9686105F02CFEEB780133EB7068688B
:105D90001022A11C381805F02BFE2E8145E76F89D3
:105DA000009A7B1E9BB293423AD1E278A37812020A
:105DB0001A43237905A81B04134362796C68120601
:105DC0001A43EB6800920392211D0C22049305F004
:105DD000C7FC0120260004A940421036FFF7E2FE6E
:105DE000013F012F17D1009A0B232861824200D076
:105DF0004CE704221C49200005F0FAFD042203A907
:105E0000686805F0CDFBE968039AFF23914200D151
:105E10003CE7F73B3AE73100FFF7C4FE1036DFE717
:105E20000923B742A4D831E7009BB34200D9FCE66E
:105E300007232BE7022329E7032327E7062325E788
:105E40000A2323E7FFFE00003C3DFF1F0000011175
:105E5000FFFF00005048593601FF0000FFFF00110E
:105E600002FF000034F00040483DFF1F10B5034C16
:105E70000B000122210000F06BFA10BD2D60001113
:105E80000B8870B506000D000224162B11D92B00CB
:105E90000322094900F05CFA041E0AD1074B2A8844
:105EA0001B88191C934200D9111C300089B200F0E4
:105EB000EFFA200070BDC04659600011DE5EFF1F82
:105EC00010B54A780400013A0B000220012A07D8D5
:105ED0000A78002A04D005222000024900F038FA8E
:105EE00010BDC046876000110A7810B50B00040091
:105EF0000220002A04D007222000024900F028FADC
:105F000010BDC046336100110A7810B50B000400C3
:105F10000220002A04D009222000024900F018FAC9
:105F200010BDC0469961001110B5034C0B000B2247
:105F3000210000F00DFA10BDC961001110B5034C2D
:105F40000B000D22210000F003FA10BD3B6200118E
:105F500010B5034C0B000F22210000F0F9F910BD21
:105F6000956200110A7810B50B0004000220002A87
:105F700004D011222000024900F0EAF910BDC04609
:105F8000A5620011002310B51322190000F0E0F9FA
:105F900010BD000010B5034C0B001722210000F0CB
:105FA000D7F910BDF7620011002310B519221900AE
:105FB00000F0CEF910BD000010B5034C0B001B2201
:105FC000210000F0C5F910BD31630011F7B58489D7
:105FD0000D0006000121002C22D000238268D35638
:105FE0001778002B1EDA0C2C1AD90C3CA4B213190A
:105FF00040880093230002F086FE431E9841013042
:106000007B06DB0F6B703F23013C1F40A4B228705E
:10601000AF70AC80002C07D0B3680133AB600021B7
:106020000800FEBD0020EBE7AC60F8E70B780370DA
:106030004B8843704B881B0A83700B79C370042014
:1060400070470420022B06D10020537811781B02E0
:10605000009A0B43138070470B8803700B881B0A50
:106060004370022070470420009983420AD153787C
:1060700010781B0203430B80D37890781B020343F4
:1060800000204B807047F8B50D004B7801240021AB
:10609000461C03702B788B4201D82000F8BD6B782A
:1060A000B01C4F1C012B10D1890069184B880222AB
:1060B00033704B88B9001B0A7370691805F060FAD9
:1060C00004360434A4B2F9B2E4E7122359436B183E
:1060D0005A88043132705B8810221B0A7370691869
:1060E00005F04EFA12361234ECE770B5049D140038
:1060F0001E00052B01D8042070BD637812781B02A6
:1061000013432B80E378A2781B02134302226B8097
:106110002A71211D681D063E05F032FAB2B22A81AD
:10612000E92AE8D82800A11D0A3005F029FA002044
:10613000E2E7002310B50A789A4201D8900010BD1A
:106140009A008A185488013304705488DBB2240AF8
:106150004470948884709288120AC2700430EAE70E
:1061600010B51100029C062B04D004201022142B21
:1061700001D010BD022222714B7808781B02034324
:106180002380CB7888781B02034363800431601D31
:1061900005F0F6F90020ECE710B50C788B780431A7
:1061A0005C43E4B203702200013005F0E9F9601CA1
:1061B00010BD0420022B06D10020537811781B0259
:1061C000009A0B431380704710B50C000A88023107
:1061D00005F0D6F9208810BD70B504000D000498B4
:1061E0001100012B01D8042070BD167852781202DC
:1061F000324302800200F13255701470E125002C08
:1062000000D10C35023B9AB24280AA42EBD802314F
:10621000043005F0B5F90020E6E704200099834238
:106220000AD1537810781B0203430B80D3789078FF
:106230001B02034300204B80704710B50C000A88F6
:10624000023105F09DF9208810BD000070B50121D4
:106250001E000420049C0E400B4218D1CB40DDB23E
:106260008D4214D90A49DBB2098899420FD3230021
:10627000EE331D703300580011184978165C09027E
:10628000314301332152D9B28D42F4D8002070BD80
:10629000543DFF1F10B50C000A88023105F070F95B
:1062A000208810BD10B50C788B7804315C43E4B2C3
:1062B00003702200013005F063F9601C10BD10B5B9
:1062C00011000298032B01D8042010BD14785278D5
:1062D000043B120222430280CA788C7812022243C5
:1062E00042809AB28280EB2AEED80431063005F063
:1062F00047F90020E9E710B50C000B8803700B8804
:106300001B0A43704B8883704B881B0AC3708A88B2
:106310000430063105F034F9A088043080B210BD95
:106320000420012B03D100201378009A13707047CA
:1063300010B50C000B8803700B881B0A43704A8849
:106340000230043105F01CF96088023080B210BDC3
:10635000F0B589B003931E4B029242000700D05A59
:10636000019102F020F81325061E2DD0029B012476
:106370000370019B002B04D0001903999847001962
:1063800084B26B461B7A5BB2002B0FDA1021380007
:1063900002F01CFB1925002813D130003219E1B29C
:1063A00002F066FC051E0CD10C34A4B2042304AA2E
:1063B000380005A993800696948101F0AFFD051E73
:1063C00002D0300005F064FA280009B0F0BDC046E4
:1063D000DC5EFF1F70B505000C0000280CD000200B
:1063E000814209D010222000044905F0C9F801209B
:1063F0002B7823736B78637370BDC0462CBD00117E
:10640000F0B506000D0017001C0085B002291BD056
:106410000020102907D1022B07D0102B03D115E043
:106420000020102C08D005B0F0BD69463800FFF7F9
:10643000D1FF2A0069460BE069463000FFF7CAFF2A
:1064400022006946380004E0022BE9D12A00390015
:10645000300005F045F9E6E7031CF02800D9F023E9
:10646000032008499AB2013A0B80D317034006492A
:106470009B189B100B80D30F04499B185B100B805B
:106480007047C046583DFF1F563DFF1F543DFF1F3C
:10649000034B1B888B4202D3024B4000C152704712
:1064A000583DFF1FDC5EFF1F014B4000185A70472C
:1064B000DC5EFF1F1722014B1A807047DC5EFF1F56
:1064C00070B505000E2005F073F9041E13D0D0231B
:1064D000037000230622837007494570033005F0DE
:1064E0004FF8064B2100DA8A62811B7E2373044B2E
:1064F000187805F00DFA70BDF85EFF1FE85EFF1F0B
:10650000A83DFF1F262803D8024B4000C05A704701
:106510000148FCE75A3DFF1FFFFF000070B5060071
:106520000C00094D1C220021280005F081F9074BC1
:106530001E70074B1C7005F03BF80123002801D0AA
:10654000002312202B7070BDE85EFF1FA83DFF1FC7
:10655000095FFF1F70B505000D4C0800E260A160E7
:1065600010220021656005F0B3F9012803D1102144
:10657000A06802F058FD10220021280005F0A8F9BB
:10658000012803D11021606802F04DFD70BDC046A6
:10659000E85EFF1F70B5041E05D1002903D0062256
:1065A0000D4804F0EDFF0D4B1D78012D11D1002C8D
:1065B00005D102221A7005F01BF9280070BD0022D7
:1065C0001A70074B1B78FF2BF7D02000FFF778FFDE
:1065D000F3E70025F1E7C046F85EFF1FE85EFF1F06
:1065E000A83DFF1F030010B5002801D1002010BDF9
:1065F00000780B4A002803D15988D1821B79137681
:106600001378022BF2D10023984200D10333137088
:10661000044B1B78FF2B01D0FFF752FF0120E6E768
:10662000E85EFF1FA83DFF1F002911D000280CD0F5
:106630004B79012803D140225242134303E03F2209
:106640001340032802D001204B7170474022F4E729
:106650000800FAE770B5094D0100287800280BD032
:10666000074C0622200004F08BFF21002878FFF75A
:10667000DBFF200005F0A4F970BDC046085FFF1FD6
:10668000E25EFF1F00290AD0012808D13F224B7982
:106690009343C02B03D0403B5A425341981C704750
:1066A00070B5174D06002B78FF2B15D00A2005F08A
:1066B0007FF8041E10D0D0230370C83B8370114BA9
:1066C00011491B784670C3700622043004F058FF4D
:1066D0002100287805F01CF90C4B1B78012B0DD1FB
:1066E0000B4B1B68002B03D09B68002B00D09847F6
:1066F000084B04211878084A05F022FA70BDC046FC
:10670000A83DFF1F085FFF1FE25EFF1F045FFF1F22
:10671000305FFF1F345FFF1F60EA0000014B986885
:106720007047C046E85EFF1F014BDB681868704782
:10673000E85EFF1F074B10B5DA681368013313607A
:10674000054B1878FF2803D08021C90105F098F87F
:1067500010BDC046E85EFF1FA83DFF1FF7B50E0045
:1067600002F0C8F8051E1CD00E4B06621F78002FE1
:1067700000D10778AB791020019305F019F8041EB9
:106780000FD0D0230380C73B8370019BE91DC370EA
:106790000622043004F0F4FE21003800E66005F023
:1067A000B7F8F7BDA63DFF1F014B18787047C046EC
:1067B000085FFF1F054B002805D1054B1A78054BD4
:1067C000002A00D1014B18007047C046F85EFF1F39
:1067D000085FFF1FE25EFF1F014B58687047C0460D
:1067E000E85EFF1F024B1868431E9841C0B2704715
:1067F0000C5FFF1F421E03000120152A03D9FF3B37
:106800005A425341D8B27047F0B51C0000230E0025
:1068100085B0039002920B70029A934201D300203C
:1068200019E0E55C5A1CD2B2002DF8D0029851193B
:106830008142F4DC0233DFB2A35C18000193FFF75E
:10684000D9FF002807D0013D019A0399EBB23370BC
:106850008A4202D1E01905B0F0BDDB19DBB2DBE7FB
:1068600010B50C0002F09EF803001220002B03D09C
:106870002100588804F0ACFF10BD000070B50E4D2B
:1068800084006359002B15D0186A002801D004F049
:10689000EFFE2B59586A002801D004F0E9FE2B596D
:1068A000986A002801D004F0E3FE285904F0E0FEC5
:1068B00000232B5170BDC046185FFF1F1C4B70B5E5
:1068C00004000E00150099420AD11A4B1B68002BD8
:1068D00001D1122070BD1B68002BFAD09847F9E750
:1068E000154B994215D1134B1B68002B0AD01B681E
:1068F000002B07D09847002804D1104B1C70104B78
:106900001D70E7E729002000FFF7AAFF0028E1D16A
:10691000F3E7080001F0EEFF0028DAD00378032047
:10692000A342D7D12900300004F052FFD2E7C0467D
:10693000FEFF0000145FFF1FFFFF0000115FFF1F3D
:10694000105FFF1FF7B50400808801F0D3FF00251A
:10695000A84203D00578A08802F008F81C4E3378CE
:10696000002B1FD0AB421DD11A4B28001978FFF71E
:1069700077FF002818D000233370A3790820A77868
:10698000A688019304F014FF011E0DD0D0230370DC
:10699000CA3B8370019B477086808371280004F096
:1069A000B7FF01E0002DE8D1A0880B4B8200D3583F
:1069B000002B01D0FFF762FF1721A088FFF768FDC9
:1069C000A08801F027FDA08801F0FEFDF7BDC046BC
:1069D000115FFF1F105FFF1F185FFF1FF0B587B02B
:1069E0001D000CAB1B88070001930DAB1B88142006
:1069F00002930EAB1B88160003930FAB1B8800910C
:106A0000049310AB1B88059304F0D2FE041E1AD029
:106A1000D0230370CB3B47708370C67006222900D9
:106A20000430002D11D004F0ABFD019B21006381E7
:106A3000029B0098A381039BE381049B2382059B17
:106A4000A37404F065FF07B0F0BD04F0F1FEECE7BD
:106A5000F7B5009308AB1B8807000C200D0016004B
:106A6000019304F0A5FE041E13D0280001F042FF9C
:106A700000280FD00078D0232370C93BA370009B5F
:106A800021002381019B6770A580E680638104F06B
:106A90003FFFF7BD014B1878EDE7C046A83DFF1F4B
:106AA00013B5040064890389C2888188C078009482
:106AB000FFF7CEFF13BD000010B5044C206800287E
:106AC00003D004F0D5FD0023236010BD1C5FFF1F21
:106AD000A122F0B5818892004A43384B384F1B6899
:106AE00004009B189D2292009B18827989B01A603D
:106AF0003B68002B5FD01D78324B1B68002B04D005
:106B00005B68002B01D00020984726000836310032
:106B1000E079FFF7B7FD237DE0710200E078049390
:106B2000638A29000393238A0293E3890193A3884C
:106B300000933300FFF752FFE378002B0BD1E2897B
:106B4000A379A18802920196E2792800009201229D
:106B500001F0DAFEE0703B68002B20D0FFF7ACFFBD
:106B6000194D287800281AD0184B1978FFF778FEAD
:106B7000002814D02B78E67808200793A78804F023
:106B800017FE011E09D0D0230370CA3B46708370E4
:106B900087808671079804F0BBFE00232B701721B5
:106BA000A088FFF775FCA08801F034FCA08801F0F4
:106BB0000BFD09B0F0BD064B9DE7C0463409FF1F31
:106BC0001C5FFF1F305FFF1F115FFF1F105FFF1F64
:106BD000A83DFF1FF8B5070008000E0001F08AFE6F
:106BE000041E18D02620FFF78DFC051E00D1257845
:106BF000062004F0DDFD041E0DD00021062204F065
:106C000017FED0232370C23B21006770A370A680BB
:106C1000E8B204F07DFEF8BDF0B585B001930AAB93
:106C20001B78070002930BAB1B7808000D00009245
:106C3000039301F05FFE061E22D0102004F0B8FD81
:106C4000041E1DD01022002104F0F2FD2620FFF7C3
:106C500059FC002800D13078D0232370C13BA370A9
:106C6000009B21002372019B67706372029BA580C9
:106C7000A372039BC0B2E3720C9BE36004F048FE76
:106C800005B0F0BDF7B50D00019001F033FE071E11
:106C900020D00E2004F08CFD041E1BD02620FFF710
:106CA00031FC061E00D13E78D0232380C53B06224E
:106CB000A370F91DE01C04F063FC019B2A006381B2
:106CC0000123DD401A401D40210022736573F0B29C
:106CD00004F01EFEF7BD0000F0B585B00290100074
:106CE0000D0017000A9E039301F004FE041E31D02C
:106CF000029B002B2ED1039B02795B0724D5122324
:106D000013430422002E08D10B99002905D10C99B8
:106D1000002902D10D9900291AD01A430D9B227126
:106D2000002B00D0C9E0002E00D1CFE0002D00D014
:106D3000CCE0606A002801D004F09AFC1C213000ED
:106D400004F0EEFD606205E002239A430E33D7E7BC
:106D500093432371654BBA00D458002C00D1AAE0AC
:106D6000002E10D0236A002B03D11C2004F0E0FC7D
:106D700020625E4BBA00D358186A002803D01C2248
:106D8000310004F0FDFB0C9B002B12D0574CBB00D4
:106D90001D596B6A002B03D1162004F0C9FC6862F0
:106DA000BB00E358586A002803D016220C9904F05F
:106DB000E7FB0D9B002B11D04C4DBC006659B36A0C
:106DC000002B03D1142004F0B3FCB0622B59986A55
:106DD000002803D014220D9904F0D2FB380001F0F2
:106DE00089FD051E67D0414BBA00D358002B62D0F5
:106DF0001A6A3420002A00D11C389A6A002A01D06D
:106E0000143080B20B9A002A01D01C3080B25B6A29
:106E1000002B01D0163080B204F0CAFC041E4AD008
:106E20001822002104F004FD2620FFF76BFB0190DF
:106E3000002801D12B780193D0232370029B2000DE
:106E400063700A23294EA370039BBD00A371AB5945
:106E5000A780196A1830002905D01C22A06004F010
:106E60008FFB200034307359996A002907D0030042
:106E700014221433E060029304F082FB02980B9B0F
:106E8000002B08D003001C221C330B9920610293B5
:106E900004F076FB02987359596A002903D0162230
:106EA000606104F06DFB6B462100187904F030FD41
:106EB0003800FFF7E3FC05B0F0BD10220D9B0D99E3
:106EC0001B69A018236204F05BFB2CE70B9B002BD3
:106ED00000D13FE7012D00D03CE7606A002801D0D7
:106EE00004F0C6FB1C210B982AE7C046185FFF1F61
:106EF00010B5044C2068002803D004F0B9FB00232F
:106F0000236010BD0C5FFF1F0B4B07B51A68002AEA
:106F100001D100200EBD6946531C012012780731B3
:106F2000FFF772FC0028F4D002780123100018400B
:106F30001A42EED0EEE7C046285FFF1FF0B51F4FA4
:106F400001203B6887B0002B25D09B78059300F08B
:106F5000B3FB002821D00A20FFF7D4FA04000B204D
:106F6000FFF7D0FA164B05001E78731E9E413B6852
:106F7000F6B2191DD878FFF757FB3B682900DA7A7B
:106F8000043303929A790193029200903300200017
:106F9000059A04F06DFC07B0F0BDFFF7B5FF0028BF
:106FA00005D00620FFF7AEFA04000720D8E7082036
:106FB000FFF7A8FA04000920D2E7C0460C5FFF1FC4
:106FC000085FFF1F70B50A4E040033780D00FF2BD9
:106FD0000DD0042004F0ECFB011E08D0D023037078
:106FE000CE3B45708370C470307804F091FC70BD66
:106FF000B83DFF1F70B5040006200D0004F0D8FB5B
:10700000011E0AD0D0230370CD3B8370054B447022
:107010001B688580187804F07BFC002C01D0FFF7FA
:1070200067FF70BD0C5FFF1FF8B5264F06003B6879
:107030000D001124002B05D10522234B1B78134290
:1070400002D112242000F8BD204A10241268002A20
:10705000F8D01278002AF5D0DB0719D52B789A1EC4
:10706000012A1AD80C2004F063FB1324386000288E
:10707000E8D000230A22437029000670023004F091
:107080007FFAFFF75BFF041E0AD0FFF731FFD9E755
:1070900000F012FB0028E1D1E4E7002BE2D0D0E7BA
:1070A0000B4B1B78032BCDD11D20FFF72BFA094B7F
:1070B00018800028C6D0084B04211878074A04F02D
:1070C0003FFDBFE70C5FFF1F095FFF1F285FFF1F2A
:1070D000085FFF1F065FFF1F345FFF1F60EA0000AD
:1070E000F7B50193194B14001A78052306000F0019
:1070F00012201A4221D0012920D1154B1D68002DE4
:107100001BD002201F2C18D8002C02D0019B002B72
:1071100013D0104B1F221E706E1C0021300004F093
:1071200087FB01992200300004F02AFA3100200088
:107130002C70002F06D004F01BFCFEBD064B122065
:107140001D68DCE704F07CFAF7E7C046095FFF1F23
:10715000285FFF1FB83DFF1F245FFF1FF8B50F4ECC
:1071600012243368002B17D01B780F3C834213D1B5
:1071700000250B4F0221387804F032FB094B042123
:1071800038781D8004F02CFB074B28001D803368E5
:107190005C7004F015FB04002000F8BD0C5FFF1FBD
:1071A000345FFF1F205FFF1F065FFF1F70B50128C0
:1071B00023D11B4C2388002B03D01A4A1578002DAD
:1071C00007D0194B1B68002B02D01878FFF7C6FFB9
:1071D00070BD3B2B02D93C3B2380F9E7134E0221C3
:1071E000307804F0FDFAFA222388920002215A43F3
:1071F000307804F095FC2580EAE70B4B1B68002BE8
:10720000E6D00B4B1B785B07E2D5084B02211878C0
:1072100004F0E6FA0022024B1A80FFF769FED7E776
:10722000205FFF1F045FFF1F0C5FFF1F345FFF1F06
:10723000095FFF1FF8B51E4D2868002803D004F031
:1072400017FA00232B601B4E3068002803D004F08F
:107250000FFA00233360184F05243B7818002040B4
:10726000234221D0154800F02BFA3B78234213D05B
:10727000202004F05DFA2860002813D0202200218D
:1072800004F0D6FA202004F053FA041E306005D032
:107290002022002104F0CCFA002004E0286804F049
:1072A000E7F92C601320F8BD00F00AFAF4E7C046B5
:1072B000285FFF1F245FFF1F095FFF1FAC3DFF1FFB
:1072C00010B50A4C23681A1E0ED0002808D10130D0
:1072D000587004F075FA002805D02368002B02D0FE
:1072E0000021FFF787FE0122100010BD0C5FFF1F79
:1072F000F7B5274E050033680191181E21D05C7840
:10730000244F012C30D1FFF7FFFD002825D02000AD
:10731000FFF7F8F80400412814D91F4B0221187810
:107320001E4A04F00DFC1E4B3C3C1C8002223368BC
:107330005A703B78002B14D128000199FFF75AFEB0
:107340000120FEBDFA2292004243002AEED0124BE9
:107350000221187804F0E4FBE8E7FFF7D3F8020015
:10736000F3E700233B70EBE73B78002BE8D10320E9
:1073700004F01EFA011E08D0D0230370CC3B4570E8
:1073800083703368187804F0C3FAFFF7B1FDD7E7CC
:107390000C5FFF1F045FFF1F345FFF1F60EA0000E8
:1073A000205FFF1F10B51749838802008B4220D051
:1073B00011D815498B4217D0144900205B1899B297
:1073C000012907D8926811785A425341D8B2FFF781
:1073D000F9FD012010BD0E4A00209B1807229BB228
:1073E0009A424041C0B2F5E783681878FFF768FF1A
:1073F000F0E7836899785A78090218781143FFF703
:1074000077FFE7E70A20000006200000F8DFFFFF13
:10741000AFDFFFFF014B18707047C046B93DFF1F3B
:1074200010B5064C207001F041FA207804F090F875
:107430000521207800F062FD10BDC046345FFF1FBB
:107440000BB273B50D00002B00DBC4E0884B18783D
:1074500004F04EFB041E0ED00378912B0FD0A22B0C
:1074600000D1A1E0834B1878FF2852D0210004F00E
:107470004FFA00284DD180200002684076BD437845
:107480000F2B76D013D8052B70D00E2BEAD1808825
:10749000794B98422BD8794B98421BD8784B98421D
:1074A000E0D1A3681878591CFFF774F838E03E2B38
:1074B000D8D18378032B74D06CD8012B6ED0022BDB
:1074C000D0D1704B1B68002B23D05B68002B20D0E1
:1074D00098471EE06C4BC0180C28C3D804F038FA4B
:1074E0001DC2C2150BC20B0B0B3223C23C00674BF3
:1074F000C0180728B6D8664B1B68002B09D01B683C
:10750000002B06D0200098470AE0A3681878FFF700
:10751000C7F8200004F014F9ADE7A068FFF762F89F
:1075200000289FD0F5E7A3681B78002BF1D0554BBE
:107530001B68002BEDD01B68002BEAD021005548BA
:107540009847EDE74F4B1B68002BE2D01B68002BE0
:10755000DFD021005048F3E7504B1B68002BD8D0F8
:107560005B68002BD5D021004348E9E7FFF7EAF933
:10757000CFE780884A4B984203D04A4B984200D0CC
:1075800070E7464B1B68002BC3D05B68002BC0D054
:107590002100D5E7153B012BBBD963E7FFF798FA2C
:1075A000B7E7FFF77DFAB4E73F4B1B78042B07D111
:1075B00000236A4613800179408800F0C5FCA8E7E3
:1075C000364B1B68002BA4D05B68002BA1D00100B8
:1075D000364898479DE7012421420AD0294B1B6871
:1075E000002B04D05B68002B01D0002098470120BD
:1075F00043E78B070AD5264B1B68002B04D05B683A
:10760000002B01D020009847022036E704212800F3
:1076100008400D4200D131E7254E3388002B21D0A0
:10762000013B9BB23380002B1AD1FFF7DBF8002817
:107630000AD0204B1C70164B1B68002B04D05B68D3
:10764000002B01D020009847FFF7C6F8694601F0EB
:1076500001FD6846FEF7FEFF1D20FEF753FF308058
:1076600004200AE7024B187804F0BAF8F8E7C0469D
:10767000345FFF1FB93DFF1F0E20000001200000F6
:10768000091000002C5FFF1FFEDFFFFFAFDFFFFFD1
:10769000305FFF1F0C2000000B200000145FFF1F55
:1076A0000D20000013200000095FFF1FFFFF0000F6
:1076B000065FFF1F045FFF1F10B501F09BF910BDAF
:1076C000014B18607047C046305FFF1F0B880020D9
:1076D000162B01D817230420014A13807047C04697
:1076E000DE5EFF1F00207047074A030011888142B9
:1076F00007D091880020994202D1013080001018F3
:1077000070470020FAE7C0463C5FFF1FF0B58F7856
:1077100006000D00C5B01E2F15D1FFF7E5FF051EB1
:1077200003D10024200045B0F0BD00223B00310011
:10773000C078009200F0B2FB0400A81C00F0D2FB5D
:10774000FF23EB70EEE7264B062403931B78FF2BF9
:10775000E8D0182FE6D87B08224A013BDB000292D2
:107760009A589446002ADDD0029AD3185B68002B01
:10777000D8D00878002802D14B78012B02D10624FA
:10778000122FCFD107AFAB88697800976446AA68FB
:10779000A047041EC6D1AB78029A5B08013BDB0010
:1077A000D318390030005B689847041E0BD1AB78C2
:1077B000042BB6D0039A310010782200009700F015
:1077C0006DFB0400AEE76A78002AABD1AA7805A960
:1077D0003B88087130000A704B80FEF747FBA0E73A
:1077E000BC3DFF1F3CBD00111D4B37B50500984245
:1077F0000BD000290AD1FFF777FF002805D11948DF
:10780000FFF772FF002800D0058037BD01291AD18B
:10781000FFF76AFF041EF8D001235B420380A378C0
:10782000FF2BF2D0FE2B07D00023E0781422009328
:1078300029001E3300F032FBA01C00F053FB012393
:107840005B426380E1E70229DFD1013901F0BEF834
:107850000028DAD12800FFF747FF041EDFD1D4E764
:10786000FEFF0000FFFF0000022210B5074B52424E
:107870001A80074801325A809A80DA8000F07EFA36
:10788000044801F025F8002010BDC0463C5FFF1FF2
:107890000D770011E97700110388F7B50400002B7C
:1078A00002D102252800FEBD426802211378254836
:1078B0005268FEF7A5FD00282ED0234F01253A88F7
:1078C000002AEFD0802321885B0201259B1A994270
:1078D000E8DC0C2003F02CFF061E31D03B88228808
:1078E0009C4600231800019561469DB2491989B252
:1078F000AA421BD8002801D062443A8000233000FD
:10790000082208C0210003F03BFE104A1368002B38
:1079100013D100251660C5E76268022113780C4870
:107920005268FEF76DFD0028C7D1BAE760681D01F7
:107930004019418101330198D6E71A001B68E6E738
:107940001325AFE7AABD0011BA3DFF1F385FFF1F27
:10795000A8BD0011014B18707047C046BC3DFF1F09
:1079600014230A0010B51A40194204D00122102134
:1079700001F048F810BD4B06F9D4012088434000BF
:10798000F8E710B514008B0604D50122102101F090
:1079900039F810BD08230A001A40194202D14BB22F
:1079A000002B0FDA102101F02DF8002808D0230059
:1079B000F2331B78002BECD0F1342378012BE8D183
:1079C0000020E6E703208907FAD4E2E7F0B51F00BC
:1079D000184B85B01C68019002910392002C27D1AE
:1079E000200005B0F0BDA5683301ED186B89019A40
:1079F000934211D3029A93420ED8002F04D10A9BCE
:107A0000002B10D12C00EBE73B002978039A686823
:107A1000FEF7F6FC0028F2D10136B6B2A388B342D5
:107A2000E1D82468DAE7A3680A9A5B891380E9E75A
:107A30000026F3E7385FFF1F37B50C000A88498836
:107A40000123914217D3002A15D0651D23792A00FE
:107A500002210A48FEF7D4FC102300280BD023791A
:107A60006188208800242A000094FFF7AFFF0A23D2
:107A7000A04200D0230018003EBDC046AABD0011A0
:107A800013B50A0008884988012388420BD80028CA
:107A900009D00024137905320094FFF797FF0A23D9
:107AA000A04200D02300180016BD13B50A000888B4
:107AB0004988012388420BD8002809D00024137973
:107AC00005320094FFF782FF0A23A04200D0230072
:107AD000180016BDF0B58BB003904A8808880E00D8
:107AE0000123824255D3002853D00023012704AC40
:107AF00023700022718813000092FFF767FF051EB4
:107B00003ED02078002835D12B78022B18D1677011
:107B10006A8983000130E31880005A806968022274
:107B2000201803F02DFD23780133DBB22370042BE2
:107B300019D93B006889013080B2002BD9D01FE0F1
:107B400002236370122358436A89231804305A8031
:107B500069681022201803F013FD23780133DBB28B
:107B60002370002BE5D10C4A6B899B185A42534174
:107B7000DBB2DFE76378012BE4D12B78022BC7D08F
:107B800022780A23002A04D021000398FEF798F9EE
:107B9000002318000BB0F0BD0100FFFF0F4BF0B544
:107BA00004001868002816D083685D89A54207D8AC
:107BB0008288AE18B44203DA12019A18934201D1B6
:107BC0000068EFE71E005F891036A74204D1002944
:107BD00000D00D801800F0BD3300EFE7385FFF1FC5
:107BE00070B505000C0008880021FFF7D7FF0300DF
:107BF0000120002B04D022002800197AFFF7C1FED3
:107C000070BDF7B50C00002501902300EE331B7802
:107C1000AB4201D800200AE06B00E65A0021300098
:107C2000E718FFF7BBFF002802D126800130FEBD18
:107C3000017A0198FFF794FE002802D03B88238048
:107C4000F5E70135EDB2E0E710B504000888002142
:107C5000FFF7A4FF03000120002B03D02000197AB6
:107C6000FFF77EFE10BD0000054B1B68002B01D105
:107C7000180004E09A6852898242F6D198887047C9
:107C8000385FFF1FF0B50E27002687B0039302ABC5
:107C9000FF183E8005001F4B40891400984207D012
:107CA0002B78013000976A6880B2FFF78FFE0600DC
:107CB00002212B7818486A68FEF7A2FB00280FD033
:107CC0006C892000FFF7D0FF002802D0013C041986
:107CD000A4B2039B002B00D01C80300007B0F0BD85
:107CE00002212B780D486A68FEF78AFB0028E7D14D
:107CF00002212B780A486A68FEF782FB002807D029
:107D0000002EDED03B88A342DBD17489013CDFE743
:107D10006C89DEE7FFFF0000AABD0011A8BD0011BD
:107D2000A6BD001110B50C00FFF7DEFC0300022019
:107D3000002B0AD0002C00D023609B781720FE2B4C
:107D400003D00138FF2B00D1002010BD73B50D000A
:107D500001A904001600FFF7E5FF172805D0002E43
:107D600004D129002000FEF727F976BD0122102159
:107D7000200000F047FE0028F3D0F6E7014B186022
:107D80007047C046485FFF1F37B56B469D1D010019
:107D900004000222280003F0E3FC2B88B02B0ED154
:107DA0002379122B09D12300FA331B78012B06D13A
:107DB0000121608800F0E0F801E01B2BF8D037BD0E
:107DC00010B5054B0421187000F098F8FFF74CFD32
:107DD000FEF770FB10BDC0464C5FFF1F0020F0B5E2
:107DE0000BB20F0087B0834234DA274B187803F0C8
:107DF0007FFE051E2BD00378A02B25D103AE3100CA
:107E0000FEF7E4F8041E0BD1B378DB0724D51F4B33
:107E100006341B68002B03D03100688898470400A3
:107E2000A868002801D003F033FD002C08D1184ABF
:107E3000039B1340174A934206D0B3781B2B03D001
:107E40000121688800F098F8280003F079FC802070
:107E50000002784007B0F0BD0F4B1B68002B10D01C
:107E6000310068889847041EDAD07378002BD7D188
:107E7000B27801A90A704B800C716888FDF7F6FF93
:107E8000CEE70624F1E7C0464C5FFF1F445FFF1FAB
:107E900000FFFF0000011200485FFF1FF7B50190CF
:107EA000FC200D0017001E0003F082FC04001320CC
:107EB000002C12D0B02320002370089BF42267709E
:107EC000658026710830002B08D0190003F058FB9C
:107ED0002100019803F01CFD0020FEBD089903F06D
:107EE000A7FCF5E710B5041E06D00078FD2803D8DE
:107EF00003F0B6FDFF23237010BD00000A1F93B2EC
:107F000010B504000220032B05D882400020024B4C
:107F1000D1529B189C7010BD6C5FFF1F0B8870B511
:107F2000043B04000D000220032B0BD8012120008C
:107F300000F04CFD03001420002B03D0290020008A
:107F400000F0DEFB70BD000007B51300034A00928D
:107F50000A00012100F02CFC0EBDC04685810011F5
:107F600007B5019203220092024B0A00122100F091
:107F700049FC0EBD0382001107B56B4601AA1180B2
:107F80000449D88008780633012802D1190003F08B
:107F900047FD07BD4D5FFF1F0C4B10B51870002348
:107FA000FF210B4A1380138193819380094A5380E8
:107FB0001370517293819372D174D3821375517778
:107FC00003F0B6FD00F0FCF910BDC0467C5FFF1F5A
:107FD0006C5FFF1F4E5FFF1FF0B58DB06B4600203A
:107FE00003910C229B5E834200DBB0E05D4B18786E
:107FF00003F07EFD051E00D1A4E00378902B00D095
:108000009DE006AF01004688380000F013FA796859
:108010000400002900D19CE03B88052B6ED13B89F0
:10802000032B1CD905AC200000F0A2F86288172AA7
:1080300061D83989131D994231D179682378043187
:108040000291D90738D5607800F08EF9071E06D066
:10805000002303712378012B08D0132B23D0A868A9
:10806000002800D178E003F013FC75E062880299E3
:1080700009A800F0A6F80290380000F08BF909AAD0
:108080002378387A0192002231000092029A00F09F
:1080900012F9380000F064F9029B002BDFD03000A9
:1080A00000F080F9DBE70378032BD8D162880299CE
:1080B00009A800F0D6F8DEE7122B13D1029909A81F
:1080C00000F0B5F8021EEAD127498B88002BC6D0F4
:1080D000887909A92378019161780091310000F035
:1080E000EAF8BCE7002302AA93833000617809AA6A
:1080F000FFF72AFFB3E71D4B0993F6E7042B02D0E5
:108100009A1F012AABD8184A043B9B00995A0029B0
:10811000A5D0D218907831003A0000F0AEF80028CF
:108120009DD13B88042B03D001213000FFF724FFB1
:10813000012C04D1A868002801D003F0A9FB280075
:1081400003F0FEFA8020039B0002434018000DB0AC
:10815000F0BD012800D182E701213000FFF70CFFBC
:10816000EDE7C0467C5FFF1F6C5FFF1F010017003B
:108170000B7803704B784370CB788A781B021343DB
:10818000438070470A88030002700A88120A42700E
:108190000A88012A06D14A8882704A88120AC27067
:1081A0000420704702208242FBD14A8804309A7032
:1081B0004A88120ADA708A881A718A88120A5A71F1
:1081C000EFE710B50400012082420CD94B780A7801
:1081D0001B0213432380834206D1CB788A781B028B
:1081E00013436380002010BD022BFBD1CB788A782B
:1081F0001B02134363804B790A791B021343A3804C
:10820000F0E70B8803700B881B0A43704B88837060
:108210004B881B0AC3708B8803718B881B0A4371C0
:10822000CB888371CB881B0AC37108207047030079
:108230000120082A14D14A780878120202431A80D1
:10824000CA788878120202435A804A790879120261
:1082500002439A80CA798879120202430020DA80A8
:10826000704710B504000120022A05D100204B7888
:108270000A781B021343238010BDF8B506001020B6
:108280000F00150003F094FA04000120002C0ED01A
:10829000A0230C22290023806780201D002D07D0F9
:1082A00003F06EF92100300003F032FB0020F8BD2E
:1082B00003F0BEFAF6E7F7B51E00009008AB1420F5
:1082C00017001D78019103F073FA041E12D0A22347
:1082D0000370019B47704380099B057146710C2216
:1082E0000830002B07D0190003F04AF9210000984C
:1082F00003F00EFBF7BD099903F09AFAF6E737B5DC
:10830000041E0FD04388002B0CD00025C1881323F6
:10831000007A172201950095FFF7CDFFFF236580B6
:108320006372257037BD000010B50C4904004A88FF
:10833000002A09D08B89002B05D00020CB8A02228D
:10834000834201D010BD012213000A2043430020C4
:108350004032C854C81842800472F3E74E5FFF1FD2
:108360000023438003707047094B00211A0010B5A9
:108370005C88002C06D01C79844203D10A234B432D
:10838000D01810BD01310A330329F1D10020F8E7DC
:108390004E5FFF1F10B50400407A03F061FBFF231E
:1083A000637210BD7047043010B580B203F010F94D
:1083B000002803D00421494203F082F910BD0000D7
:1083C00070B50025104CA0682580A581A580A84225
:1083D00002D003F05DFAA56000250C4C0C4B606DDB
:1083E0001D80230058331D70A84202D003F050FABC
:1083F000656500256068002801D003F049FA013561
:1084000008340A2DF6D170BD1460FF1FB85FFF1F3E
:108410000860FF1F70B5041E09D1054D2880A88192
:10842000A880A868002802D003F032FAAC6070BDC2
:108430001460FF1FF0B54B8885B0019300234360A3
:108440000A7905000F00022A00D07BE0CA88032ABF
:1084500017D98B685E7819783602DC78D8790E43A4
:1084600099781B7A24021B020C43034353495BBADD
:108470000B80331D93421ED1042C04D0631F022BAA
:108480000ED9012015E0019A4D4B1201D35A002B51
:1084900006D00198FFF7BEFF4A4A13690133136102
:1084A0000421B8682E812C80494203F009F96860E4
:1084B000002005B0F0BD434D042C06D0631F022BF5
:1084C0000FD9EB680133EB60DBE7019A3C4B1201FB
:1084D000D35A002B05D00198FFF79CFF2B6901337D
:1084E0002B61374B30000293019B029A1B010193D1
:1084F000002301998C468B52130063449C800393A4
:108500009E81FFF750FF039B041E986016D0042144
:10851000B868494203F0D4F8FA880100043A200010
:1085200003F02EF80199029AFB888A5A043B9B18A3
:10853000029A8B522B6801332B60A2E7AB6901339F
:10854000AB619EE71E4B0293019B1E01029BF35AF7
:10855000002B2DD002998C19A068002828D0012A60
:1085600026D1FA889B189BB27352A189994217D3DE
:108570009B1AC018B96803F003F8029BA289F35A4A
:10858000934200D07DE700222B81A3882B80A36833
:108590006B60029BF2520B4A53680133536070E7E1
:1085A000084A9368013393600198FFF733FF68E747
:1085B000044A536901335361F6E7C0467E5FFF1FEB
:1085C0001460FF1F845FFF1F70B5051E15D10B4C93
:1085D0000B4B1880230058331870606D002802D0B0
:1085E00003F056F96565250050356068002801D014
:1085F00003F04EF90834AC42F7D170BDB85FFF1FED
:108600000860FF1FF0B51700A12285B0920001930A
:108610004243394B06001B680C009B18D933FF33CB
:108620001D78FDF741FF0430854204DD3000FDF781
:108630003BFF0430C5B2BD4207D33A0000213000F1
:10864000019B03F095F805B0F0BD2900380003F058
:10865000F7F82300C6B250331E700393019B290024
:108660006365380003F024FACBB20293002B02D0EA
:10867000039B01361E7000262300503303931B78A2
:10868000B34204D8606D002831D10020DBE7029AA4
:108690002800002A04D0013B1000B34200D028007B
:1086A000F700E719387003F01BFA786000280ED045
:1086B0003A78019902F064FF019A3B780136D318A9
:1086C0000E4A0193D369F6B20133D361D4E7039B19
:1086D00018706065A74205D1084A1320D36A013398
:1086E000D362B0E7606803F0D3F80834F2E703F030
:1086F000CFF800236365C8E73409FF1F845FFF1FBD
:10870000F7B50D0007000421686802F0D9FF2B8936
:10871000040003702B891B0A43702B8883702B88FD
:108720001B0AC3702E8902250436F6B2F42E15D822
:108730001B4B9F4214D10C2003F03AF81135011E57
:108740000CD0902303708E3B0371043B4380154B88
:108750008460C680187803F0DBF800252800FEBD91
:108760005C237B43104AD3180093583301931B7842
:10877000002B0FD10300320038000099FFF742FFB1
:10878000019B05001B78002BE8D13800009903F00D
:108790005FF8E3E7054A0725536A01335362DDE7D3
:1087A000FEFF00007C5FFF1FB85FFF1F845FFF1F9D
:1087B000F0B587B0009017200F0016000193FFF767
:1087C000F2FD1325041E19D00C98031E02D0019946
:1087D000201D9847030AE370052302AAA070043005
:1087E000908127700098667003A993800494FFF726
:1087F00087FF051E02D0200003F04AF8280007B0CA
:10880000F0BD0000F0B587B01F000CAB1B780391E2
:10881000059301210DAB06001C78049200F0D6F8F8
:108820001425002821D02000FFF77EFD0135041E0D
:108830001BD01149059B0A7803700132D2B2131E76
:10884000C68001D101231A000B7022713000049BF5
:1088500003990097FFF7ACFF051E09D12300210003
:108860000648074A093303F02BF9280007B0F0BD8A
:10887000002363802370F8E7805FFF1FFF820011F1
:1088800030750000F8B505000E00064C064F236851
:10889000002B02D03100280098470434BC42F6D1A6
:1088A000F8BDC0462460FF1F3860FF1F0123064A41
:1088B0005B425380002313715362044A1360536078
:1088C0009360D360136170473860FF1F2460FF1FFF
:1088D0000200002310B506499C000859002801D168
:1088E000625010BD0133052BF6D11320F9E7C046C5
:1088F0002460FF1F034A5388181A434258414042DC
:10890000104070473860FF1FF0B585B002930AAB86
:108910001F780CAB1B88009008000E000192039397
:10892000FFF7E8FF05001120002D1BD10E48FFF7CF
:10893000E1FF04001520002C14D006220B99A7712A
:10894000E01D02F01DFE019B30002371029B2900F7
:108950006371009B66802370039B6562E381FFF770
:1089600091FF280005B0F0BDFFFF000010B5FFF734
:10897000C1FF04000220002C12D060880121FFF703
:1089800081FF606A002801D002F072FE28220021D7
:10899000200002F04DFF012300205B426380207124
:1089A00010BD000030B5074A074C55880100137808
:1089B0000020A54204D05B1A59424B415842104056
:1089C00030BDC0463860FF1FFFFF0000084A10B5E9
:1089D00001230C00904208D0FFF78CFF031E04D047
:1089E000037923405A1E9341DBB2180010BDC046E4
:1089F000FEFF0000024B1879431E9841C0B2704739
:108A00003860FF1F70B504000D001600FFF772FFFD
:108A1000002804D10D4B9C4200D0143070BD416A37
:108A200003790520002907D012221A40102A02D10A
:108A30000520002EF2D10F20DB06EFD5897E0C2019
:108A4000A9428941494249420840E7E7FEFF000048
:108A5000030010B5002800D110BD0348034A418827
:108A60009142F9D09847F7E73860FF1FFFFF0000F9
:108A7000002330B5C45CCD5C6C40D4540133102B62
:108A8000F8D130BD0F23002210B5C45C640022432E
:108A9000CA54C25CD209013BF7D210BD02000100EA
:108AA00010B52032103102F07BFF10BDF0B58BB055
:108AB0000390102005931700049102F039FE0090F6
:108AC000102002F035FE009B13240190002B05D0EE
:108AD00000280CD11324009802F0CAFD019B002B42
:108AE00002D0180002F0C4FD20000BB0F0BD102031
:108AF00002F01EFE0600102002F01AFE13240500EC
:108B0000002E00D1AEE0002819D01022002102F082
:108B10008FFE32002900039802F042FF041E0ED19E
:108B200033787F2B51D830000099FFF7ABFF009BC3
:108B30001B787F2B53D801990098FFF7A3FF3000D3
:108B400002F096FD002D02D0280002F091FD002CCD
:108B5000C1D1102002F0ECFD0600102002F0E8FD6B
:108B60000290002E7CD0002878D03A000F322300EB
:108B70000125121105D00F333B4015B25A42534123
:108B80001BB26A1E1201002B33D0049BD2B298187C
:108B90000099029AFFF76CFF013D1022002130007E
:108BA00002F046FEADB2049F2D017D19AF4242D0C6
:108BB000002C33D0300002F05BFD029B002B00D173
:108BC00089E7180002F054FD85E729003000FFF71F
:108BD00059FF28002549009AFFF74AFFA7E7290017
:108BE0000098FFF74FFF28002049019AFFF740FF48
:108BF000A5E70F210F4004998A18D9B28F4208D9EE
:108C0000D15C06A819540133102BF6D1029A0199B0
:108C1000C0E7791A48424141C901F2E73900300002
:108C200006AAFFF725FF3200039806A902F0B8FE56
:108C300010370400BAE7002CBCD13000029906AA14
:108C4000FFF716FF320006A9039802F0A9FE0822DA
:108C500004003100059802F093FCABE71324A9E768
:108C60001324AAE7002800D06EE733E7B0BD001157
:108C7000F0B58BB00F0016000225009000283FD001
:108C8000002A3DD00B1DDBB21800029302F050FD0C
:108C90001135041E34D0FDF747FD05003A00009958
:108CA000201D02F05DFEEBB20393E3702B0CDBB2F0
:108CB0002F0A00936370FFB22B0E2370A7700193ED
:108CC000FDF72CFD1022010006A802F049FE21004C
:108CD000029A04AB06A8FFF7E9FE051E0DD1039B1F
:108CE00008223370009B04A9B370019B7770F37066
:108CF000301D02F035FEFDF71DFD200002F0B8FC2E
:108D000028000BB0F0BDF0B58FB00D00149E03909D
:108D100004920593002A03D1022420000FB0F0BD75
:108D2000002EF9D00398FFF7E5FD1424071EF4D0B8
:108D30007278337812021A43B3781B041343F27823
:108D400012061A43036A0192934201D30133E3D11D
:108D5000002D03D03B7901249B07DED5082200219A
:108D600006A802F065FD059B13240433DBB218004E
:108D7000029302F0DDFC051ECFD0059A0499043061
:108D800002F0EEFD04223100280002F0E9FD390076
:108D9000102210310AA802F0E3FD2900029A06AB66
:108DA0000AA8FFF783FE041E0FD1082206A908A80F
:108DB00002F0D6FD0822311D08A802F091FC01281E
:108DC00007D101990398FDF7C9FC280002F050FC77
:108DD000A3E70124F9E7000070B51C4C05002368E7
:108DE000181E10D0002D14D11A78002A0CD1981C0E
:108DF000083202F0C5FB02F0BBFB0135002808D1A8
:108E000023681D70012070BD0A331800082202F08B
:108E1000B7FB2368002BF5D0122002F0C9FC061E18
:108E20000DD0C12321680370457002311022023039
:108E300002F0A6FB23683100587802F069FD206833
:108E400002F016FC00232360DCE7C0466060FF1FD1
:108E5000F8B504002020FDF755FB0D4EA700BB59C7
:108E60000500002B0DD000280BD0D878FF2809D1A1
:108E700008492A000C55F35907480333611802F0DA
:108E80001FFEF8BD290002F06BFE0028F0D1F8E7C4
:108E90007C60FF1F6460FF1FA9A0001170B5064D24
:108EA00084006359002B05D0D87802F0D9FDFF2249
:108EB0006359DA7070BDC0467C60FF1F70B5060054
:108EC0008CB00C00150000213022684602F0B0FC86
:108ED00031001022684602F043FD1D2021000322CC
:108EE000684402F03DFD6846FFF7D8FD2D210400DF
:108EF00003222800694402F033FD20000CB070BD4D
:108F0000F0B50700160097B001931CAB1D78302216
:108F10001EAB00910AA800211C7802F089FC1022E7
:108F200039000AA802F01CFD1022002102A802F05C
:108F30007FFC0722310002A802F012FD072202ABDB
:108F40009818631E9C41019902F00AFD02AB9C73C4
:108F50002B005A1E934102AAD3730021102206A8A7
:108F600002F066FC06221D9907A802F0F9FC1A20FF
:108F700002ABC01806221F9902F0F2FC10220099E1
:108F80000EA802F0EDFC102202AB0EA908781C78A6
:108F9000013A6040D2B2087001330131002AF5D1A4
:108FA0000AA8FFF77BFD102212A904000EA802F008
:108FB000E7FA102206AB0EA908781D78013A68403E
:108FC000D2B2087001330131002AF5D10AA8FFF7A7
:108FD00065FD044310222098E4B212A902F0C0FCFF
:108FE000200017B0F0BD70B50E0014008CB0010069
:108FF000102268461D0002F0B3FC3100082204A8CC
:1090000002F0AEFC2100082206A802F0A9FC684686
:10901000FFF744FD04001022280008A902F0A0FC7C
:1090200020000CB070BDF8B506000D000024371903
:10903000AC4200D3F8BD02F0EBFC030A3B70631CAA
:10904000DBB201379D4203D90234F054E4B2EEE7BB
:109050001C00EDE773B506000C000225002819D0AE
:10906000002917D0032101A8FFF7DDFF6B469A798D
:109070003F231A40013313436A463000937101A91C
:109080002200FFF71BFF051E04D10322E01C01A9EB
:1090900002F076FA280076BD03785807DA08C00F88
:1090A000D20080009B0710439B0F1843C0B270474B
:1090B00007230B40C908C9000B4303707047000029
:1090C00070B50400FFF7EAFE134DA4006359002BAE
:1090D00021D0186A002801D002F0CAFA2B59986EE4
:1090E000002801D002F0C4FA2B59D86E002801D014
:1090F00002F0BEFA2B59186F002801D002F0B8FA1E
:109100002B59586F002801D002F0B2FA285902F00A
:10911000AFFA00232B5170BD7C60FF1F0E4B800007
:10912000C35870B50C00002B0FD09D68002D0CD0DB
:109130002B78201D0B706B784B70A97CFFF7B8FF64
:109140002B7E23726B69E36070BD1022002120002A
:1091500002F06EFBF8E7C0467C60FF1F014B186011
:109160007047C0467860FF1F074A0300800082589E
:1091700010B5002A06D0D088984203D1012901D128
:10918000FFF79EFF10BDC0467C60FF1FF0B5264E66
:1091900095B087000B93BB590500099112200A92E4
:1091A000002B31D0D888FFF7A5FB04001420002C39
:1091B0002AD0280010A9FFF7B1FFBB591E781D6AFD
:1091C000002E23D00895FDF7EFFA07000020FDF7E9
:1091D000F1FA0790A379E61D069310AD0CA9089843
:1091E00000F0E2FA0EA9280000F0D7FA0B9B0A99CA
:1091F0000493069B09980293079B0396019300979B
:109200000EAB0CAAFFF77CFE15B0F0BDFDF7CCFA53
:1092100006903000FDF7CEFAE31DA779079310AB57
:1092200006000893DAE7C0467C60FF1F30B50C4C9F
:1092300085002A59030085B00120002A0ED01800AD
:109240006946FFF76BFF2B591A78D888054B002A1F
:1092500000D1054B6A46072100F0D9FB05B030BDAF
:109260007C60FF1F9B970011A997001130B5094C36
:109270008500295985B010226846253102F080F911
:109280002A591121044BD0886A4600F0C0FB05B072
:1092900030BDC0467C60FF1F4598001130B5094CB9
:1092A0008500295985B010226846353102F068F9E9
:1092B0002A591121044BD0886A4600F0A8FB05B05A
:1092C00030BDC0467C60FF1F83980011F7B54D4F3D
:1092D00086001020F4590D0002F02AFAF35920629A
:1092E000186A132200286CD0033A29009C6802F007
:1092F00047F9F3591A780192002A58D11E6A227D43
:10930000317B944651400122019F114201D16746B1
:109310001740217D914339432175377B4F40BC462F
:1093200060460027800701D44F0817400121022022
:109330008F40227D82433A432275377B5740BC469B
:1093400060460027400701D497080F400420227D83
:10935000BF0082433A432275627D002794466046EF
:10936000727B42400A4201D167460F400121627D73
:109370008A433A436275777B5740BC466046002774
:10938000800701D457080F400220627D7F0082438E
:1093900017436775767B00227E40760701D4BA08B2
:1093A0000A400426617D9200B1430A4362756A78DF
:1093B000002A08D06278002A05D005220533DA7722
:1093C00000221000FEBD04222979114205D1A17CA2
:1093D000114202D10533033AF1E7019A21782C7842
:1093E000002A02D10A002100140018220429E8D81A
:1093F000042CE6D805206043034A05331218525C5A
:10940000DDE7C0467C60FF1FC0BD001110B50A003B
:109410001121024B00F0FBFA10BDC046DF9800118D
:109420000B0030B587B001AD2B806B4604001100F6
:10943000981D082202F0A4F82A000B212000024BFC
:1094400000F0E5FA07B030BD0799001110B50A0029
:109450001121024B00F0DBFA10BDC0465B990011F0
:1094600013B50B0011006A4613706B460400062208
:10947000581C02F085F86A4608212000014B00F0D4
:10948000C6FA13BD7B99001110B50A001121024BD9
:1094900000F0BDFA10BDC046CB9900117FB50500A4
:1094A0000B4BAA00D4580800002C0FD0666F237F06
:1094B000E28821780396266F0296E66E0196A46EE6
:1094C0000094FDF709FC2800FFF7FAFD7FBDC046B8
:1094D0007C60FF1F10B51721FFF7E0FF10BD0000F3
:1094E00070B50A000D00064B0221040000F08FFA4F
:1094F000060029782000FFF7D1FF300070BDC0467C
:10950000AB98001170B586B000236A46137083686B
:1095100004001D78681E0A2859D801A902F0B8F87D
:10952000060633373B3F43474B4F5300180000F0CC
:1095300042F9062312284BD000281BD16088FFF780
:10954000D9F90823002813D04279002A47D1264BA5
:109550001A78072312070BD5244B1A680723002A11
:1095600006D01668002E03D0290001AAB0470300D8
:109570006A4613706B461B786088002B2AD1FFF770
:1095800067FC06B070BD180000F06CF9D4E7180055
:1095900000F087F9D0E7180000F093F9CCE7180045
:1095A00000F0ADF9C8E7180000F0C3F9C4E71800EF
:1095B00000F0F6F9C0E7180000F0F6F9BCE7180073
:1095C00000F013FAB8E7180000F013FAB4E7072325
:1095D0006A46137069466088FFF782FFD1E705236A
:1095E000012AC5D1024BB8E7095FFF1F7460FF1F56
:1095F0007860FF1FF8B52C4F8600F35904000D006A
:10960000002B40D0DA8882423DD15A78062A33D1E5
:109610001A78002A2ED0012099681A6A097D014221
:1096200006D0157B054203D007225A700120F8BDF1
:109630000220014204D0157B054201D00922F4E743
:109640000420014204D0127B024201D00B22ECE73D
:10965000164B1B68002BE9D05B68002BE6D020007E
:109660009847BB5900215B78122BDFD12000FFF710
:1096700015FFDBE70E4BECE7112A04D1002900D0DF
:1096800032252900F2E7002D08D12000FFF732F93A
:10969000002803D01023027913430371210028000E
:1096A000FDF798FAC2E7C0467C60FF1F7460FF1F99
:1096B0007860FF1F70B50E4E8500AB590400002B7B
:1096C00013D01B78002B11D10A4B1B68002B04D040
:1096D0005B68002B01D02000984773595B78122BF0
:1096E00003D100212000FFF7D9FE70BD024BECE74B
:1096F0007C60FF1F7860FF1F7460FF1F094B8000B4
:10970000C3581020002B0CD01A6A002A09D09B687D
:10971000002B06D0127A1B7E101C9A4200D9181C0E
:10972000C0B270477C60FF1F70B503000D001400CD
:109730000220002A30D000292ED013700B78081D8B
:1097400053704B789370FFF7A7FCE0700120022163
:109750002B7A23716B7B034063716A7B0A4013434E
:10976000042263716E7B1640334363716E7BF6088F
:10977000F600334363712B7B0340A371287B0140C8
:1097800000200B43A371297B0A401343A3712A7B5A
:10979000D208D2001343A37170BD10B50A000100B6
:1097A0000120FFF7C1FF10BD10B50A000100022023
:1097B000FFF7BAFF10BD70B506000C000220002EA6
:1097C00030D000292ED07378201D0B70B3784B70E9
:1097D000F178FFF76DFC01223579257271794B1014
:1097E000080013409340104003438810104080004D
:1097F000C9080343C9000B436373B1794B100800D8
:109800001340934010400343881002409200C9085F
:109810001343C9000B4321202373FCF773FE8542D9
:1098200001D2122070BD2220257AFCF76BFE854202
:10983000F7D823781820042BF4D86378012BF1D8BB
:109840000020EFE7030010B50220002909D0002B0B
:1098500007D00322481C0A7019000D3201F090FE57
:10986000002010BD03000222080010B5002B06D016
:10987000002904D00E32591C01F082FE0022100093
:1098800010BD030010B50220002909D0002B07D01D
:109890000422481C0A7019000C3201F071FE0020ED
:1098A00010BD10B5FFF7DEFF10BD03000220002938
:1098B00006D0002B04D0052200200A701B784B70C4
:1098C000704703000220002B08D0002906D05B78E7
:1098D00000200B70013B082B00D9183070470300A3
:1098E00010B50220002909D0002B07D00622481C01
:1098F0000A7019000A3201F043FE002010BD10B5B5
:10990000FFF7B0FF10BD02000B00022010B50029C8
:109910000ED0002A0CD007211970118859701188B7
:10992000090A997011180822D81C01F029FE00209C
:1099300010BD03000A00022010B5002B0CD0002936
:109940000AD099785878090201431180901CD91CDB
:10995000082201F015FE002010BD030010B5022002
:10996000002909D0002B07D00822481C0A701900D2
:10997000921801F005FE002010BD02000B0002202D
:1099800010B500290BD0002A09D0092119701178CF
:1099900018185970511C062201F0F2FD002010BD6C
:1099A00010B5FFF75FFF10BD02000B00022010B5DD
:1099B000002A09D0002907D0517819701118062201
:1099C000581C01F0DDFD002010BD030010B5022081
:1099D000002909D0002B07D00A22481C0A70190060
:1099E000063201F0CDFD002010BD10B5FFF73AFFA3
:1099F00010BD02000B00022010B5002A06D000297D
:109A000004D018005178FFF753FB002010BDF0B5CB
:109A100085B017001E006A460623050008009181E4
:109A20009380FEF7C0FC1324011E02900CD0380076
:109A3000B047041E05D1280001A9FEF76FFA041EE5
:109A400002D0029801F024FF2800FFF701FA20005D
:109A500005B0F0BDF0B504008BB0019115000021F8
:109A6000102202A801F0E4FE334EA700B8590028E6
:109A70003CD0C388A34239D10378002B36D1427839
:109A8000062A18D102000100553235310C3006ABE0
:109A9000FFF7A9FA002829D12000FFF72FFE0200C6
:109AA00006A902A801F06CFD200002A901F020FE29
:109AB00001200BB0F0BD816E002917D00B8A112A4E
:109AC00028D19D420ED101981231093A01F008FEC9
:109AD000012807D1BB5920009D6EFFF70FFE29001A
:109AE0000200DEE732212000FFF7D8FC2000FEF75D
:109AF00001FF061E1BD0416A002918D00B8AAB4219
:109B000015D108220198123101F0EAFD01280ED189
:109B1000716A0AE09D42E9D108220198123101F0F0
:109B2000DFFD0128E2D1BB59996E8A7EB9E720009A
:109B300001F0B6FFBCE7C0467C60FF1FF0B56B4D7F
:109B400087007E5985B0337802900393002B00D0B4
:109B500087E0B368346A01937078062817D1012230
:109B60001B7D134202D0217B114218D102221342E5
:109B700002D0217B114251D10422134203D0237B16
:109B8000134200D08BE0019B5A7DEB5991E00738DE
:109B90000428F8D801F07CFD032E42678300B36EE1
:109BA000002B03D11C2001F0C3FDB066EB599C6E65
:109BB000002C1CD010220021200001F039FE029858
:109BC000FFF79CFD01002000FFF72DFA01F020FFB8
:109BD0002082200008211230FFF725FA0298FFF7B3
:109BE0008DFDA076EB592100D888FFF70FFC0822E5
:109BF000EB591CE0B36E002B05D01A00198AF088CF
:109C00001232FFF70DFC0222019B197DEB59114224
:109C10003DD0207B10423AD0073208E0F488FCF7B0
:109C2000DBFD01002000FFF711FC0A22EB595A70FE
:109C3000029B9C002A595378073B042B11D8D088EB
:109C4000FEF758FE00284ED0C3895A08D21828497A
:109C5000029B0298CB542B5941180433254801F03C
:109C60002FFF05B0F0BDFCF79FFD030001208342EC
:109C700001D100200393EB59DE88FCF79BFD03998B
:109C800002003000FFF7ECFB019AEB59117D042232
:109C900011420CD0217B114209D00B22C7E7F68874
:109CA000FCF73CFD01003000FFF7EEFB6BE7019A8B
:109CB000527D01210A4204D0607B084201D00C226F
:109CC000B5E702210A4204D0607B084201D00E228F
:109CD000ADE704210A4204D0627B0A4201D010227F
:109CE000A5E71222A3E7FA225200B0E77C60FF1F2B
:109CF0008060FF1FB3A0001110B5064B1A78042333
:109D0000100018401A4200D00348FFF727FA00203D
:109D100010BDC046095FFF1FC03DFF1F70B50400A6
:109D2000FFF7D4FA051E43D12000FFF77FFA234E38
:109D3000A400A0598268937CDB0708D50321036A3D
:109D40001B790B40012B02D1017F0B430377431D8D
:109D5000D97F8B1E022B0DD8022900D00121C0888B
:109D6000FCF790FF042133591A7F59700A431A7780
:109D7000280070BD01290CD102231022437000215C
:109D80000C3001F055FD305910213530FFF74BF9FB
:109D9000EEE70529ECD10223D118437010220C30D4
:109DA00001F0EEFB04233259117F0B431377EAE7EE
:109DB00008251828DCD1053DDAE7C0467C60FF1F86
:109DC000F0B58BB0059143887E4F9E00F459150085
:109DD0000493002C15D1012902D000200BB0F0BD56
:109DE000101D57781678FFF757F9EB683200029389
:109DF0002B7A0499019300903B002000FCF70CFFA4
:109E0000EBE7E388049A934201D00820E6E7237841
:109E1000012B00D1D4E0059B581E092800D9CFE0C2
:109E200001F036FC05CE0A29CC506C859AB2290087
:109E30000498FFF773FFD1E7200029001022453076
:109E400001F09EFBB9594B78042B02D1013B4B70BA
:109E5000C3E70B000A00253335320C310498FFF7B5
:109E600095F90498FFF702FA0522431E9841BB5961
:109E7000C0005A70B2E7200029001022553001F0CE
:109E80007FFB049B4F4C9D00295904980A0006ABA8
:109E900055320C31FFF77AF929591022453106A8BD
:109EA00001F01EFC012808D10498FFF7F7F905908E
:109EB000002804D106222B595A7005988EE70823F2
:109EC0000593FAE763780C2B7AD1E36E002B03D16C
:109ED0001C2001F02DFCE066BB59D86E00286FD025
:109EE0001022290001F04CFBBB590498DC6EFFF7EF
:109EF00005FC0D22A076BB595A706EE7E06E002873
:109F00005ED063780D2B5BD12B8808220382A91CBD
:109F1000123001F035FBBB599A68517D0222114283
:109F200026D0186A407B104222D00C32E4E76378D6
:109F30000E2B45D1236F002B03D1162001F0F8FB27
:109F40002067BB59186F002803D01022290001F0A8
:109F500017FB0F22BB59CFE763780F2B30D1206F4F
:109F60000622691C103001F00BFBBB599A68517D29
:109F70000422114203D0196A497B1142D5D1002134
:109F80000498FFF78BFA28E7636F002B0DD0BB59BD
:109F9000586F0028F3D01022290001F0F1FA0122B5
:109FA000BB5952425B6F1A61E9E7142001F0C0FB14
:109FB000BB5960675B6F002BE9D126E72978DFE7A3
:109FC00007200BE77C60FF1F10B5064C207001F0E6
:109FD000DFFC06212078FDF791FF0348FEF778FCAF
:109FE00010BDC0468F60FF1F6991001100200BB2A9
:109FF00070B50D00834216DA264B187801F078FD13
:10A00000041E0DD00378922B0ED0A02B37D0224BFC
:10A010001878FF283AD0210001F07AFC002835D1C9
:10A0200080200002684070BD43780E2B0BD03E2B81
:10A03000EDD18378052B12D0082BE8D18179808867
:10A04000FFF7D8FA08E0154B82889A42DFD183687F
:10A050001878591CFEF7C0FE002817D1D7E7104B1F
:10A060001B785B0712D50F4B1B68002B0ED09B682B
:10A07000002B0BD0C289811D80889847ECE7FFF741
:10A0800041FAA068002801D001F002FC200001F094
:10A0900057FBC5E78F60FF1FB93DFF1F1820000069
:10A0A000095FFF1F7860FF1F10B50078FFF712FAF5
:10A0B00010BD10B50078FFF7FDFA10BD0C23434327
:10A0C000084A10B59B185A68002A03D0012901D10B
:10A0D000904710BD9B68002BFBD00029F9D1984711
:10A0E000F7E7C046AC60FF1F01238340094A10B563
:10A0F000946B1C439463506B98435063D46B200063
:10A100009843012901D120001843D063116B0B4300
:10A11000136310BD00800040F0B500240127154BEB
:10A1200085B0DA6B144E03921A6C0192DA64019BCB
:10A13000E3403B4217D0039DE5403D400295E5B228
:10A1400002992800FFF7BAFF316A736A002908D024
:10A150003900002B01D0029979402800FFF7C4FF95
:10A1600001E0002BF9D101340C36172CDFD105B0FA
:10A17000F0BDC046008000409060FF1F064B0121EB
:10A180005A68C2400A4204D01B68C3401800084005
:10A1900070471B6DF9E7C046008000400122064B66
:10A1A0008240002903D0D9680A43DA607047D96831
:10A1B0009143D960FAE7C0460038004030B5032427
:10A1C00044430F4BE25C1B199C785D7801232D1BE7
:10A1D0000135AB40013BA340A140DB430C001228FA
:10A1E00007D808499200521811681940214311609C
:10A1F00030BD054A11680B4023431360F8E7C046A1
:10A2000007BE001108F0004014F00040C21F70B5F6
:10A21000D4B20623092C0BD80125084C95400029FF
:10A2200008D00021FFF7CAFF23682B4323600023D7
:10A23000180070BD2368AB43F8E7C0460038004003
:10A24000214BF0B51B185B78022B21D1032444432A
:10A250001E4A1F4EA35C12199478012215008540F6
:10A26000B76B013CE4B23D43A240B563194C1228E0
:10A2700015D89B0000290CD117495B1899680A432F
:10A280009A600123205C154A834011680B431360D8
:10A29000F0BD11495B18996891439960F1E70E4B45
:10A2A00000290DD159690A435A61225C1328E8D06C
:10A2B0000123203A93400A49086803430B60E7E70B
:10A2C000596991435961F0E79060FF1F07BE001183
:10A2D000008000404CBE001100F00040A0F00040A3
:10A2E000A4F00040F8B500241B4E1C4D1C4B1B5D18
:10A2F000012B1FD1194A9269E2401A420BD0012268
:10A30000B25693402200143AD2B2022A09D8154913
:10A310004A6913434B61013402360C35172CE5D1E1
:10A32000F8BD0022B2560F499200521891680B43B3
:10A330009360F0E7022BEED1E7B23800FFF71EFF83
:10A3400001235840C1B23800FFF77AFF3800FFF709
:10A3500015FF6877DFE7C046D9BD00119060FF1F89
:10A360009160FF1F00F00040012202388240054B3F
:10A37000002903D059690A435A61704759699143CA
:10A380005961FAE700380040F8B50E0001210F00CE
:10A390008740114A0400D368FD43BB43D360831E4A
:10A3A0008B4201D8FFF7E0FF00212000FFF72EFFCE
:10A3B0000A4A0B4B5168012E05D139431B195160D4
:10A3C0005E700020F8BD2940516002221C196270A5
:10A3D0009A6915409D61F4E7003800400080004014
:10A3E0009060FF1F012210B58240074B002906D064
:10A3F00019680A431A600121FFF7C6FF10BD1968EA
:10A4000091431960F7E7C046008000400C2370B507
:10A41000002543430A4A29009B181D70094B04007C
:10A420001B185D70FFF7B0FF0123A3400649280009
:10A430000A681A430A6005490A689A430A6070BDAF
:10A44000AC60FF1F9060FF1F3480004030800040F0
:10A4500070B504000E00FF2813D003250540FFF758
:10A46000D5FF084AA3089B009B183F22ED00AA4095
:10A47000AE40196820009143314319600121FFF774
:10A480008DFE70BD18380040F8B50C244443134BC2
:10A490000500E4186368002B03D1A3681220002B89
:10A4A0001AD0022201270E4B00215B195A70280096
:10A4B0002770FFF769FF63681E1E08D0A3683E007F
:10A4C000002B04D02800FFF759FE4640F6B22800C2
:10A4D0003100FFF709FE0020F8BDC046AC60FF1F49
:10A4E0009060FF1FF7B5C420FF222B4B8000195846
:10A4F000002491433F3A0A431A508022274F5202C8
:10A50000274E1A60274B1D5D002D21D0A31E012B65
:10A5100003D80121E0B2FFF727FF012D18D11F4B0F
:10A520009B69E3402B4213D0E3B218000193FFF77D
:10A5300025FE01000198FFF755FFE3B2143B022B03
:10A540001DD801217156184A8D405369AB435361A0
:10A550003B7F002B0DD0E5B22800FFF795FF2800C8
:10A56000FFF70CFE7B7F0100834202D02800FFF73B
:10A57000A5FD01340C370236172CC3D1F7BD0121DC
:10A5800000237156F3568D40074A9B009B189A682A
:10A59000AA439A60DCE7C04600E100E09060FF1F3C
:10A5A000D9BD00119160FF1F00F0004070B50E0092
:10A5B00015000400FFF72AFF0C236343094A20001B
:10A5C0009B189D605E60FFF75FFFF021064B074A16
:10A5D0008900051E5A5002D02000FFF717FF2800FF
:10A5E00070BDC046AC60FF1F0000FF1F19A1001125
:10A5F00070B5134D07202C78002C1FD19822210014
:10A600005200280001F0D4F90123C420FF222B704E
:10A610000C4B80001C635C630B4B1C605C600B4B41
:10A62000195891433F3A0A431A50802252021A6045
:10A630000D20074A074901F063F8200070BDC046AD
:10A640009060FF1F00800040A0F0004000E100E0AB
:10A65000E5A40011E5A2001170B51D0002240C292B
:10A6600010D8094ACA40D2070CD5FBF757FF041E81
:10A6700008D1059A04992800FBF76CFFFCF7DAFD76
:10A68000FFF73AFB200070BD1210000030B50D78C6
:10A6900002232C009C43184201D02B431C000825A8
:10A6A0002300AB43284201D02B00234320241D006C
:10A6B000A543204201D01C4325002A230D701842D7
:10A6C00004D011781E3B0B43137030BD0028FCD121
:10A6D0000C2113788B43F7E7F8B51D0006AB1B88F8
:10A6E000140007AA0E000B201778002B27D10A7838
:10A6F000022A49D14A68507811780002244A084356
:10A700008018042840D800F0C3FF03121D1B23004B
:10A71000F06800F0C5FF021CC0B2B84200D93A1C74
:10A72000D2B22000F1682A8000F02AFF06E002225F
:10A73000F3681B882A8023701B0A63700020F8BD11
:10A740000622EEE701232B80F3681B782370F5E7E0
:10A75000F368002B16D008222A801A8822701A88E3
:10A76000120A62705A88A2705A88120AE2709A8895
:10A7700022719A88120A6271DA88A271DB881B0A38
:10A78000E371DBE72B80D9E701202B80D7E7C046B8
:10A7900000D6FFFFF7B516000A781D0008AB1F882A
:10A7A0000C000123022A18D14A685078117800025F
:10A7B0002B4A0843801803280FD800F069FF0225B0
:10A7C0004439E06800F06CFFC0B20723B84204D3FC
:10A7D0007B190193152B02DD0D231800FEBDE068E7
:10A7E0002A003100C01900F0CBFE6B4600209B8888
:10A7F000E268D0541B4B1B68834203D01B68834222
:10A8000000D098470023E8E70B23002FE5D1022D65
:10A81000E2D1737832781B021343E2681380114B44
:10A820001B68002BEED01B68002BEBD00120E8E763
:10A830000B23002FD1D1062DCED12A003100E068A4
:10A8400000F09EFEDEE70B23002FC6D1012DC3D101
:10A8500032787533012AC0D8E3681A70D2E7C0464F
:10A8600000D6FFFF9C62FF1F70B50C001500072883
:10A8700037D800F00DFF041436361B36242E18206E
:10A8800015290BD8184E16220021300000F0D0FFF9
:10A8900022002900300000F073FE002070BD182057
:10A8A0000229FBD11288114B1A80F6E718200829DB
:10A8B000F4D10A000E48290000F052FFEDE71820FD
:10A8C0000129EBD10B4B10780B49DA69FFF7DEFE5B
:10A8D000E3E718200129E1D1064B10780749DA6B2C
:10A8E000F4E70220DAE7C0468462FF1F623EFF1FE2
:10A8F000583EFF1FE83DFF1F103EFF1F303EFF1F69
:10A90000030010B50020DB0704D50721024A0348E5
:10A9100000F08CF810BDC04664BE0011E83DFF1F7A
:10A92000054A03001068002803D082889A4201D1AA
:10A93000806870470068F6E79464FF1F0A88030088
:10A9400008009A4204D08A8804309A4200D000203D
:10A9500070470000F8B5F22200230D4F0D4E7968C4
:10A96000050042433370994200D07B600A4C0021BD
:10A97000200000F05DFF00231A007C60AB4202D192
:10A9800000203370F8BD01332280DBB2F234F5E7EA
:10A990008C65FF1F8A65FF1F9864FF1F73B56B46A8
:10A9A00001900600684615001980FCF775FF041E2B
:10A9B00011D1002D0FD07689002E11D00C2000F07F
:10A9C000B7FE00280ED0084A0460136886808560B0
:10A9D000002B02D11060200076BD1A001B68F7E73B
:10A9E0000224F8E71324F6E79464FF1F01210022F4
:10A9F0000A4B10B549420A4C198099809A719A7095
:10AA0000084B2070012019805A60FFF7A3FF2078BF
:10AA1000FCF7A0FF0448FDF75BFF10BDA462FF1F19
:10AA20009465FF1F8C65FF1FD9AA0011022310B582
:10AA3000002802D0FFF7B2FF0300180010BD00008D
:10AA4000030010B50020DB0704D50421024A0348A7
:10AA5000FFF7A4FF10BDC04678BE0011683EFF1F7F
:10AA6000F0B50E2687B003930CAB1F8802ABF61827
:10AA70000500080031000292FDF790F80400012063
:10AA8000002C0FD03088FFF74BFF03000E20002B67
:10AA900008D05E68002E05D021002800039B029A92
:10AAA0000097B04707B0F0BD0A4B10B5984207D1E8
:10AAB0000122002352420A808B708A808B7110BD64
:10AAC000FFF73CFF0028FAD001235B4203800023FC
:10AAD0008370F4E7FFFF0000F8B5050001290AD1F3
:10AAE000134E00243388F227AB4219D028001149B5
:10AAF000FFF7DAFF06E0022904D10139FDF766FF0E
:10AB00000028EDD0F8BD3B0063437268D018D35ADB
:10AB1000002B09D03A00002100F08AFE0134E4B293
:10AB2000054B1B78A342EED801235B423380DDE75F
:10AB30008C65FF1FA462FF1F8A65FF1F10B5FFF71A
:10AB4000FDFE03000020834200D0987810BD000075
:10AB5000F0B589B01C000EAB80CB03901E8810AB03
:10AB60001B78049202930B7A0D00DB0616D42B7827
:10AB70000593022B24D00498FFF7D2FE002812D0B0
:10AB800003689C46002B0ED0029B220001932900F3
:10AB90003B00644603980096A04705E00498FFF741
:10ABA000BFFE002802D10E2009B0F0BD8368002B43
:10ABB000F9D00A222900039898470028D7D0F3E754
:10ABC0006B6858781A786B4B000210439842D2D8C1
:10ABD000043B984210D2684B984242D015D8674B3C
:10ABE000C0180128C7D80B20002EDDD1EB681A78D9
:10ABF00059683A80200028E0614BC018032800D92A
:10AC000079E000F045FD846A789E5E4B9842B2D1AF
:10AC10000B20002EC8D101233B80EB6831001B784C
:10AC200023706889013080B2FCF7B8FF3A88031EB0
:10AC30000ED0017802328A183A80428962704289C5
:10AC4000120AA27059680278E01C00F099FC06E034
:10AC500004323A8031000422601C00F0E9FD00203B
:10AC6000A2E70B20002E9FD1EB6807A91E880423C2
:10AC70003B80330A300026706370FCF78FFF051E9F
:10AC800028D004AB9A890E2304A95B183E49C668F4
:10AC9000FCF7F8FF00280BD12B783C486A6805992F
:10ACA000FBF7AEFB002803D1012304AA5B42D3814A
:10ACB0003278022A06D17168201D00F061FC3B88C1
:10ACC00002333B800E2304AA9B181B88A3701B0A27
:10ACD000E370C4E704ABDE81F4E70B20002E00D064
:10ACE00062E7E9680398FFF729FF02233B802070A1
:10ACF000000A6070B3E70B20002E00D054E7022258
:10AD0000EB681B883A8023701B0A6370A7E7E8682A
:10AD100000F0C6FCC2B203000720B24200D243E7F3
:10AD20000DD00299DBB27118994202DB921BD3B2AB
:10AD30000293029BE9681A003B8089195AE70023B5
:10AD4000F6E70B20002E00D02EE70722EB683A80B2
:10AD50001A7822705A7862705A88A2705A88120A39
:10AD6000E2701A792271DA886271DB881B0AA3719A
:10AD700075E7C046042900000228000000D8FFFF44
:10AD8000FFD6FFFF03280000FFFF0000A8BD001151
:10AD9000F0B58DB06B460020089120229B5E834267
:10ADA0003DDAA64B187800F0A3FE071E32D00378D8
:10ADB000B02B2CD10079023816281FD800F0B8FD2E
:10ADC00017001E001E001E0031001E0096001E000F
:10ADD0001D011E0052011E0073011E00CD011E0048
:10ADE00050021E001E001E008E021E00E302944B45
:10ADF00094491B8878880B80FBF742F83800FCF7F1
:10AE0000C3FF914B1B68002B01D0380098473800D6
:10AE100000F096FC8020089B0002434018000DB013
:10AE2000F0BDEE220021874800F002FD0BAA3B7B1B
:10AE30007989388900923A000D32FCF7C7FD040089
:10AE4000804B1B78002C3FD146E0804B78880593DF
:10AE50007F4B4100CB5A0BAE073BDBB232880293EB
:10AE6000002301937B4B210006930093059BFFF782
:10AE70006FFE744D002810D1069B3A8A1B889A42B7
:10AE80000BD138000599123000F02AFC002804D0BC
:10AE90002B7862899B00EB185A80162306A81B1892
:10AEA000328820007989FCF7EDFE2B7804009A00A7
:10AEB000AA1851880029C3D00133DBB22B700028B7
:10AEC00007D006A9C98A9180634A12889A42BCD8E1
:10AED00002E0012149429180002B04D05949788831
:10AEE000FBF702F88AE73E890A2479E000253E89CB
:10AEF000574B06937B88069A5B009B5A033B9D4207
:10AF000002DB002DF0D05BE0162206A812183B7B76
:10AF1000798900923A0030000D32FCF757FD059018
:10AF2000002858D04689017A7888FCF719FD041E5C
:10AF300044D1464B78880793069B4100C95A454B3C
:10AF40000439C9B206AAD28A0693029101940093E9
:10AF50000599079BFFF7FCFD041E2FD1069B39497D
:10AF60001A88931C002D26D14B807988384B4900D4
:10AF7000CB5A5119033B8B4220DD059B31485B893D
:10AF800041190B71A91C0135C9B2EDB205914519E2
:10AF90001B0A2B71059B2D490433181800F0F0FA99
:10AFA0002C4B059A1B88D318DDB22C4B9E4205D042
:10AFB0000136B6B29CE749889942D6D0002D0CD014
:10AFC000204C2800618800F043FD20702100788823
:10AFD000FAF79AFF12E7059CF0E7002C00D183E70F
:10AFE0007B78142B00D109E716493B794E800B7012
:10AFF0000C717888FAF73AFF00E7162406ABE418DC
:10B0000021003889FCF7CAFD011E00D1B7E178881C
:10B0100022880F4C45002C5B0A4D013CE4B202949F
:10B0200000240F4B01940095FFF792FD041E00D001
:10B0300014E129007888FAF777FFDFE69465FF1FAF
:10B04000583DFF1FAC62FF1FA062FF1FA063FF1FE0
:10B05000DC5EFF1F9064FF1F563DFF1FFFFF0000D7
:10B06000AE62FF1F162406ABE41821003889FCF7F6
:10B0700095FD011E00D182E178882288AE4C450002
:10B080002C5BAE4D013CE4B202947C89AC4B019444
:10B090000095FFF75DFD041E00D0DFE029007888F1
:10B0A000FAF74CFFAAE60025A44B1D803B00F633BF
:10B0B0001B78A24A78880792AB4208D99E4B128827
:10B0C0000693069943005B5A013B9A4203DB0799BA
:10B0D000FAF73EFF92E616246B00FB18059306ABC9
:10B0E000E418059B21001889FCF758FD011E03D1C7
:10B0F000059B01241E8973E77888924B2288069C61
:10B10000099343001B5B904E013BDBB2029300238B
:10B1100000960193099BFFF71BFD041E02D0059BBF
:10B120001E895DE77B88069A5B009B5A079A108808
:10B1300032881218934202DC1B1A013B33807F4C89
:10B14000023032880999001900F01AFA23883288EF
:10B1500001359B182380EDB2A8E70BAA3B7B7989C8
:10B16000388900923A000D32FCF730FC002505903A
:10B17000059B002B04D10A24002D00D16EE060E075
:10B18000059B7888197AFCF7EBFB0100041E63D15C
:10B19000694C6C4B788806940993069B4400E45AEA
:10B1A000694B063CE4B20BAE3288079302940191DE
:10B1B00000930599099BFFF7CBFC041E4CD1079B1C
:10B1C0005E491B881A1D002D30D14A80059B5B4CBF
:10B1D0005A8963191A716B1C9BB2E318120A1A710F
:10B1E000162306A832881B1879890598FCF74AFDB2
:10B1F000FF21AA1C2E1D03350B00059092B2B6B29A
:10B20000ADB2002803D006ABDB8AD9B21B0AA21864
:10B21000651911712B714C4D301D2A884949201830
:10B2200000F0AEF92B88F618B5B2A1E74988914233
:10B2300007D17A8806995200525AEB18053A9A4279
:10B24000C4DC3E4C2800618800F0FAFA207021002E
:10B250007888FAF787FED1E5002DF2D13E89BFE666
:10B26000162606ABF61831003889FCF797FC3D002E
:10B270000400FA3500282DD0037A9B060CD4002256
:10B280007B893989788800923A000C32FFF7E8FB15
:10B29000041E10D03E8915E03088FFF741FB0028DE
:10B2A0001AD08368002B17D0210012227888984783
:10B2B000041EE4D0EEE72B78002B02D17888FAF751
:10B2C00061FE00262B78002B00D097E5002C00D1E2
:10B2D00094E585E60124DDE70E24DBE7162506ABC1
:10B2E000ED1829003889FCF759FC041E47D0037A71
:10B2F0009B0611D4154A7B881188994203D01448C3
:10B30000814207D11380134BF2261D780023D9B256
:10B31000A94221D30924A1E72888FFF701FB0028CF
:10B320002FD08368002B2CD02100122278889847D8
:10B33000041EDFD092E7C046DC5EFF1FAC62FF1F39
:10B34000AE62FF1FA063FF1F9064FF1F8C65FF1F8D
:10B35000FFFF00008A65FF1F310059435468013325
:10B360006018615A0029D2D13C0008342100F22231
:10B3700000F006F921007888FAF70CFE3EE501247A
:10B380006CE70E246AE71D4B1A887B889A4231D0FD
:10B390007888FAF709FE31E5F223059851684343AE
:10B3A000CD18C95A00291FD03B7A012B0BD16C88CC
:10B3B000AB887888AA1D0094FFF752FB041E02D0C8
:10B3C00000233B722E88F2220021280000F030FA80
:10B3D00000232B80059B0133DBB20593084B0599B5
:10B3E0001B78064A8B42D7D801235B421380002C7E
:10B3F000CED0F5E5002634000596EFE78C65FF1FFB
:10B400008A65FF1F70B504000E001500FFF796FA5D
:10B41000031E08D131000548FFF790FA0300112000
:10B42000002B02D01C8000209D7070BDFFFF00002B
:10B43000F8B50B4F06003B780D001400FF2B0ED023
:10B440000A2000F0B5F9011E09D0B12303800023C2
:10B4500046800371C5800481387800F059FAF8BD40
:10B46000A93EFF1FF7B50F0008A90600088809A923
:10B470000B240988002821D10234022B1ED15578D3
:10B4800013782D021D432B008B4301937334002B43
:10B4900014D1FB68300019000093FFF74FFB019CAB
:10B4A00085420BD02A0030000099FFF7ABFF041E45
:10B4B00004D12A0030007989FFF7BAFF2000FEBDD1
:10B4C000F0B50E7885B003900AA805880120022EF9
:10B4D0000DD14C682778647824023C43054FBC4268
:10B4E00005D10398DBB201960095FFF7BBFF05B0CD
:10B4F000F0BDC04602290000034B10B51B68002BAD
:10B5000000D09847FEE7C0469865FF1F07B501A821
:10B51000FFF7F2FF044A05480021121A00F048FA2A
:10B52000F8F768F9FEE7C0469C65FF1FAC3EFF1FB9
:10B5300001B40248844601BC604700BFC9A90000AD
:10B5400001B40248844601BC604700BFB933FF1F05
:10B5500001B40248844601BC604700BF5D1700008B
:10B5600001B40248844601BC604700BF6DBC0000C6
:10B5700001B40248844601BC604700BFD91B0000EB
:10B5800001B40248844601BC604700BFE94C010099
:10B5900001B40248844601BC604700BFF928FF1F80
:10B5A00001B40248844601BC604700BFF530FF1F6C
:10B5B00001B40248844601BC604700BF5125000029
:10B5C00001B40248844601BC604700BF0D2BFF1F39
:10B5D00001B40248844601BC604700BFE92800006E
:10B5E00001B40248844601BC604700BFC530FF1F5C
:10B5F00001B40248844601BC604700BF3D1800000A
:10B6000001B40248844601BC604700BFED4A010016
:10B6100001B40248844601BC604700BFDD660100FA
:10B6200001B40248844601BC604700BF25260000E3
:10B6300001B40248844601BC604700BF75A9000000
:10B6400001B40248844601BC604700BF5522000097
:10B6500001B40248844601BC604700BFA54F010009
:10B6600001B40248844601BC604700BF055E00008B
:10B6700001B40248844601BC604700BF014C010090
:10B6800001B40248844601BC604700BFA534FF1FD7
:10B6900001B40248844601BC604700BF6136FF1F09
:10B6A00001B40248844601BC604700BFDD5201007E
:10B6B00001B40248844601BC604700BF0124000079
:10B6C00001B40248844601BC604700BF55490100EF
:10B6D00001B40248844601BC604700BFF52AFF1F41
:10B6E00001B40248844601BC604700BFCD4C010054
:10B6F00001B40248844601BC604700BF311B000012
:10B7000001B40248844601BC604700BF952BFF1F6F
:10B7100001B40248844601BC604700BF5D2DFF1F95
:10B7200001B40248844601BC604700BF6571010056
:10B7300001B40248844601BC604700BF3D4B010094
:10B7400001B40248844601BC604700BF434D01007C
:10B7500001B40248844601BC604700BF4550000068
:10B7600001B40248844601BC604700BF810E00005E
:10B7700001B40248844601BC604700BF5118FF1F56
:10B7800001B40248844601BC604700BFD130FF1FAE
:10B7900001B40248844601BC604700BF2135FF1F49
:10B7A00001B40248844601BC604700BFF30E0000AC
:10B7B00001B40248844601BC604700BF1D4D010032
:10B7C00001B40248844601BC604700BF691F000005
:10B7D00001B40248844601BC604700BF8D120000DE
:10B7E00001B40248844601BC604700BFB352010067
:10B7F00001B40248844601BC604700BF291C000018
:10B8000001B40248844601BC604700BF350E000009
:10B8100001B40248844601BC604700BF9DA90000F6
:10B8200001B40248844601BC604700BF35550000A2
:10B8300001B40248844601BC604700BF154D0100B9
:10B8400001B40248844601BC604700BF090E0000F5
:10B8500001B40248844601BC604700BF7D18FF1F49
:10B8600001B40248844601BC604700BFC51D00000A
:10B8700001B40248844601BC604700BF851F000038
:10B8800001B40248844601BC604700BF0D5201006C
:10B8900001B40248844601BC604700BFD949010099
:10B8A00001B40248844601BC604700BFC94A010098
:10B8B00001B40248844601BC604700BF456B0100EB
:10B8C00001B40248844601BC604700BF2146010024
:10B8D00001B40248844601BC604700BF1D4B010013
:10B8E00001B40248844601BC604700BF4D35FF1FCC
:10B8F00001B40248844601BC604700BF6D33FF1F9E
:10B9000001B40248844601BC604700BF3934FF1FC0
:10B9100001B40248844601BC604700BF594F010092
:10B9200001B40248844601BC604700BFF94C0100E5
:10B9300001B40248844601BC604700BF7536FF1F52
:10B9400001B40248844601BC604700BF4D2BFF1F75
:10B9500001B40248844601BC604700BF4D36FF1F5A
:10B9600001B40248844601BC604700BF4551010054
:10B9700001B40248844601BC604700BF4D1F00006F
:10B9800001B40248844601BC604700BF8D2EFF1FF2
:10B9900001B40248844601BC604700BFC9260000CC
:10B9A00001B40248844601BC604700BFE54800007E
:10B9B00001B40248844601BC604700BFB70E0000D6
:10B9C00001B40248844601BC604700BFC5210000A5
:10B9D00001B40248844601BC604700BF352DFF1FFB
:10B9E00001B40248844601BC604700BF7932FF1FA2
:10B9F00001B40248844601BC604700BFC531FF1F47
:10BA000001B40248844601BC604700BF056A0000DB
:10BA100001B40248844601BC604700BF29510100BF
:10BA200001B40248844601BC604700BFE117000032
:10BA300001B40248844601BC604700BFC56D0100E7
:10BA400001B40248844601BC604700BF8133FF1F38
:10BA500001B40248844601BC604700BF350E0000B7
:10BA600001B40248844601BC604700BF1147010091
:10BA700001B40248844601BC604700BF2124000095
:10BA800001B40248844601BC604700BF156B010049
:10BA900001B40248844601BC604700BF85520100E2
:10BAA00001B40248844601BC604700BF091B000086
:10BAB00001B40248844601BC604700BF090E000083
:10BAC00001B40248844601BC604700BFA94601009A
:10BAD00001B40248844601BC604700BFF933FF1F30
:10BAE00001B40248844601BC604700BF017F0000EA
:10BAF00001B40248844601BC604700BFF54E010016
:10BB000001B40248844601BC604700BFADAE0000EE
:10BB100001B40248844601BC604700BFB54C010037
:10BB200001B40248844601BC604700BF8B5201004B
:10BB300001B40248844601BC604700BF7918000088
:10BB400001B40248844601BC604700BF595201005D
:10BB500001B40248844601BC604700BFEDA5000067
:10BB600001B40248844601BC604700BF5147010050
:10BB700001B40248844601BC604700BFB14E0000DA
:10BB80000003010202030303040305000602070089
:10BB9000080209030A030B030C000D000E030F0338
:10BBA00010031103120313031403150216020000FD
:10BBB000B53B0011E93B001100000000020000004D
:10BBC000C6BB0011192A0F180A000000F159000025
:10BBD000FD24000041460100D97F0011ED9F0011B6
:10BBE00041740011DD7D0011B952001191AD0011B9
:10BBF000214F0011A93D0011D93E001100000000A5
:10BC0000161600000200000010BC0011F4FFF3FF44
:10BC1000D2FC0000194000110000000000000000EC
:10BC2000547579610042312E34003030313700676D
:10BC300069746875622E636F6D2F70767678005424
:10BC4000484231000200000058BC0011292A282A6D
:10BC5000272A262A252A242A0A180000E20400009E
:10BC60007102000078EC0000744000001027000012
:10BC700060F0000006640000204E0000000000009C
:10BC8000050000001F501D00023CB4000001170019
:10BC900014000000A1020000303132333435363751
:10BCA000383941424344454600000000BD5600116A
:10BCB000115700110000000002000000C4BC001178
:10BCC0006F2A6E2A1A18EAD8BC80F0FC60000000C7
:10BCD0000000000000005F066B2F363D7D077F3FB0
:10BCE000777C596E7971000001A00000000000000F
:10BCF0006410B71DC8206E3BAC30D9269041DC766D
:10BD0000F4516B6B5861B24D3C7105502083B8ED16
:10BD100044930FF0E8A3D6D68CB361CBB0C2649B3A
:10BD2000D4D2D38678E20AA01CF2BDBDFB349B5F5F
:10BD3000800000800010000000000000436000113F
:10BD4000CD76001167600011D57A0011EB6000110B
:10BD5000AB7A001161610011817A0011B3610011A9
:10BD6000497C00111B620011497C00114D620011D9
:10BD7000037C001161610011397A0011D961001151
:10BD8000E17B00110000000000000000BF62001114
:10BD9000E17B001121630011E5760011052A042AD8
:10BDA000012A002A02290328012800280118001866
:10BDB00000000000000000000000000000000087FC
:10BDC0000101020102010102010203030401030156
:10BDD000010101010303020103000D000E00100028
:10BDE000110013001401070108010A010B011C01D5
:10BDF0001D02040205020702080219021A021C02AF
:10BE00001D030103020317000201000504000807D7
:10BE1000000B0A001716001D1C0102010105040198
:10BE20000E0D011110011413011716011A19020247
:10BE300001020B0A020E0D02111002141302171652
:10BE4000030504030807030B0A030E0D0001020398
:10BE500007090A0B0E0F101112141718191A1B1FBD
:10BE600020212200D9A6001195A700110000000092
:10BE700002000000AEBD001100000000C1B40011BE
:0CBE80000000000002000000ACBD00113A
:020000041FFFDC
:1000000000000000113D0011CCBB0011C8BB001165
:10001000B85BFF1F000000000000000000000000AF
:1000200000000000000000000000000000000000D0
:1000300000000000000000000000000000000000C0
:1000400000000000000000000000000000000000B0
:1000500000000000000000000000000000000000A0
:100060000000000000000000000000000000000090
:100070000000000000000000000000000000000080
:100080000000000000000000000000000000000070
:100090000000000000000000000000000000000060
:1000A0000000000000000000000000000000000050
:1000B0000000000000000000000000000000000040
:1000C0000000000000000000000000000000000030
:1000D0000000000000000000000000000000000020
:1000E0000000000000000000000000000000000010
:1000F0000000000000000000000000000000000000
:1001000000000000000000000000000000000000EF
:1001100000000000000000000000000000000000DF
:1001200000000000000000000000000000000000CF
:1001300000000000000000000000000000000000BF
:1001400000000000000000000000000000000000AF
:10015000000000000000000000000000000000009F
:10016000000000000000000000000000000000008F
:10017000000000000000000000000000000000007F
:10018000000000000000000000000000000000006F
:10019000812DFF1FE12BFF1FC16601000000000041
:1001A000000000000000000000000000000000004F
:1001B000000000000000000000000000000000003F
:1001C000000000000000000000000000000000002F
:1001D000000000000000000000000000000000001F
:1001E000000000000000000000000000000000000F
:1001F00000000000000000000000000000000000FF
:1002000000000000000000000000000000000000EE
:1002100000000000000000000000000000000000DE
:1002200000000000000000000000000000000000CE
:1002300000000000000000000000000000000000BE
:1002400000000000000000000000000000000000AE
:10025000000000000000000000000000000000009E
:10026000000000000000000000000000000000008E
:10027000000000000000000000000000000000007E
:10028000000000000000000000000000000000006E
:10029000000000000000000000000000000000005E
:1002A000000000000000000000000000000000004E
:1002B000000000000000000000000000000000003E
:1002C000000000000000000000000000000000002E
:1002D000000000000000000000000000000000001E
:1002E000000000000000000000000000000000000E
:1002F00000000000000000000000000000000000FE
:1003000000000000000000000000000000000000ED
:1003100000000000000000000000000000000000DD
:1003200000000000000000000000000000000000CD
:1003300000000000000000000000000000000000BD
:1003400000000000000000000000000000000000AD
:10035000000000000000000000000000000000009D
:10036000000000000000000000000000000000008D
:100370000DB50011000000000000000000000000AA
:10038000000000000000000000000000000000006D
:10039000000000000000000000000000000000005D
:1003A000000000000000000000000000591AFF1FBC
:1003B000000000000000000000000000000000003D
:1003C000000000000000000000000000000000002D
:1003D000000000000000000000000000000000001D
:1003E000000000000000000000000000000000000D
:1003F00000000000000000000000000000000000FD
:08183800A069FF1F4118FF1F0A
:10184000024981F3088802F037F80000A069FF1F01
:1018500010B502F0A9F8072804D0122808D00228F1
:1018600008D010BD044A0420136B01331363F8E75A
:101870000220F6E71420F4E7845FFF1FF8B50700A5
:101880000C0026002500503630785135002804D150
:101890000300287058342370F8BD2978CA00481E08
:1018A0008141A3183800A25C5B68C9B2FFF7D0FF82
:1018B00000280DD12B78DA00A218013350602B706C
:1018C0003378044A013B3370136A01331362D8E75B
:1018D0000123DFE7845FFF1F5C234343074910B503
:1018E000C9180B0058331B78012B05D1FFF7C6FF31
:1018F000034A936A0133936210BDC046B85FFF1F6D
:10190000845FFF1F10B502F0CFF8064A01211300D3
:1019100010CB4942D967044B136002F0DDF8200078
:1019200010BDC04600E100E01000100010B504003A
:1019300002F0BAF8024B1C6002F0CEF810BDC046AF
:1019400000E100E0431E5A425341A022F0B5D2010B
:101950005B421340154D164A40019B182A18127E0F
:101960008BB00191002A1BD01A000832D46F0022DC
:10197000E6B206AFE4B294420EDC2818C369002B2D
:1019800008D0019902AA117106AA049202AA16733C
:1019900003A898470BB0F0BD1978B9540132EAE7B3
:1019A0001A7D1A7806AB01261A70E6E74462FF1F1B
:1019B00000400040F0B5254B04004001C25C85B0FA
:1019C000002A2BD01A18117E002927D0917E0029D9
:1019D00024D01179022921D11689D788D168F51B25
:1019E000ADB22A1C102D00D9102292B2BE4217D1DE
:1019F0001818012303710023C269C38003819A422E
:101A000006D06846032103730171029301A8904731
:101A10000820002C00D0192001F098F805B0F0BD86
:101A2000013C65426C41A0256442ED012C40084D0B
:101A30001B186419074D0633013A92B2AA42EDD041
:101A40001888461C1E80085C2070F5E74462FF1F62
:101A500000400040FFFF00000F220E4B10B59868B9
:101A6000104002380A280BD801F0FAFD0D0A0B0AC3
:101A70000A110A0A0A0A060002210020FFF762FF83
:101A800010BD0121F9E70020FFF794FFF8E7DB6FB5
:101A9000F6E7C046004000400F220E4B10B5986894
:101AA000104002380A280BD801F0DAFD0E0A0B0AA2
:101AB0000A120A0A0A0A060002210120FFF742FF61
:101AC00010BD01210800F9E70120FFF773FFF7E7D8
:101AD000DB6FF5E700900040564B70B51B68012B9B
:101AE00003D1554A936D0133936501F03DFE534B8D
:101AF000534A1860534B544C1A600123534A1360E5
:101B0000534A13602378002B06D0062251495248CD
:101B100001F032FF00232370504A514B10681B78AC
:101B2000C1B2002B0ED14F4CC0B223785BB2002B58
:101B30004FDB237824785BB264B21B0424021B19A8
:101B40001B1813600B1C50294ED95023464A474995
:101B50001078DBB2FF2202284BD10868444C454D77
:101B6000267890432A78964254D9227824782E7881
:101B7000023B5D10A31B6B435201D31A10335B1160
:101B80001843086001F080FF031F012B45D83A4B32
:101B90001B78002B06D0394B1B78002B02D000207D
:101BA00001F07AFEA122364B92009978354B4A43D8
:101BB0001B689B18832292009B181B78033B012B08
:101BC00003D8AF20400001F0A7FE01222E4BDA829D
:101BD00070BD237824785BB264B2FF33FF341B04FA
:101BE00024021B190138ABE7CAB2022AAED2022383
:101BF000ACE70868254C264D267890432A78964213
:101C000008D9227824782D78023B5B10641B63434B
:101C10005201B2E72378DBB2B2E70228D5D11D4BDF
:101C20001B78013B022B03D91B4B1B78022BCCD119
:101C30006C20C8E79809FF1FFC0FFF1FBC5EFF1F49
:101C4000FF3F000014100340C05EFF1F0C10034054
:101C500000100340D50BFF1F7211FF1FB40003409B
:101C60008C09FF1F680AFF1F490AFF1F94000340E9
:101C7000460AFF1F470AFF1FF908FF1F2209FF1F1F
:101C8000300DFF1F3409FF1FBC0BFF1F440AFF1F4D
:101C9000450AFF1F1C09FF1F2309FF1F10B501F094
:101CA00043FD0022014B1A8010BDC046B85EFF1FE5
:101CB00070B5244D2B68002B28D001F085FE2B68D1
:101CC000D8402B680400002B27D001F085FE2B683C
:101CD000D8401D4B1D4A9978A1239B004B431268A5
:101CE000D118D25C91239B00002A20D0CA5801321F
:101CF000CA50174B17491B680868834214D3D23B5C
:101D0000181A012A1AD0144B186070BD01F05CFE3D
:101D1000124B196801F0D8FCD3E701F05DFE0F4BC0
:101D2000196801F0D1FCD4E70D495B18E8E7CA5007
:101D30000C4B1B68DB68E418201AE4E7F530FF3031
:101D4000E1E7C0461C08FF1F300DFF1F3409FF1FCD
:101D50009C09FF1FBC5EFF1FA009FF1F1808FF1F83
:101D60002DFF3F00C45EFF1F70B504000D00282941
:101D700016D10300A433C2881B889B1A0B4A9BB25E
:101D800093420DD906006A3605223100653001F014
:101D90006BFE002804D13100200001F065FD70BD0C
:101DA0002900200001F050FDF9E7C046FE7F000049
:101DB000F8B50500012001F0D7FD134CA36AA26A13
:101DC0009342FBD1114E336001F036FD1049030000
:101DD00008601048426894460F4A17680022BC45C4
:101DE00001D24268BA1A0D4802603268AD18A422C6
:101DF000E562606A520302436262094A1278002A6D
:101E000001D00F3B0B60F8BD00F00040340AFF1F0B
:101E1000E408FF1F28100040180AFF1F1C0AFF1FBC
:101E20001C09FF1F70B580241025E405A3682B430F
:101E3000A36001F081FDA368AB43A36070BD000007
:101E4000F7B5160080221C001023D205019191687D
:101E500005000B43936000225A4BD7301A6001F003
:101E6000FBFD9D232A002F009B00EB58CA32012165
:101E70000092FC37002B01D00021009A386801F055
:101E8000CBFC2900009BCB311A784F4BD3351A601D
:101E90004B780A781B0213438A7812041A43CB78D2
:101EA0001B061343494A1BBA13604B790A791B027C
:101EB00013438A7912041A43CB7931001B0613436A
:101EC000434A1BBA13606B782A781B021343AA7823
:101ED00012041A43EB781B0613433E4A1BBA1360E5
:101EE000019A330213433C4A13603C4B22001B1BF4
:101EF0009C4603293DDCB3089A0013005142B21AF4
:101F0000032A46D1354AE018511A827840781204E3
:101F100000020243E05C043302430A600022FF2B0C
:101F20004BDDF0222E4B12011A600F222D4B1A604E
:101F30002D4A1368002BFCD00023224A2749136046
:101F4000091B321D0B191B68043A180A23706070B4
:101F5000180C1B0EA070E3700434002AF2DC8022FF
:101F600010213B68D20501333B6093688B4393603B
:101F7000F7BD6346D578981893782D061B042B433C
:101F8000157804392B43557804322D022B43036016
:101F9000AFE7022A0AD1114AE05C511AE2185278DE
:101FA000120202430A6004339BB2B7E7012AB5D19B
:101FB0000A4A521AE15C1160F5E7084959180A60AB
:101FC0000433ACE7000004403C0004403800044007
:101FD00034000440300004400C0004400001044080
:101FE000040004401000044014000440F7B515003C
:101FF00080221C001023D2050091916807000B433A
:1020000093600023654AD730136001F025FD9D23BE
:102010003E009B00F9583B00CA363200FC330029D1
:1020200000D07FE0586801F0F7FB390032785C4B54
:10203000CB311A604B780A781B0213438A78AC467E
:1020400012041A43CB78281D1B061343554A1BBAAA
:1020500013604B790A791B0213438A7912041A43DD
:10206000CB791B061343504A1BBA13604B7A0A7A8A
:102070001B0213438A7A12041A43CB7A21001B06EF
:1020800013434A4A1BBA1360009A2B021343484A6F
:1020900013602200474B1B1B0093009BCE785B18FC
:1020A00001938B7836061B0433430E780438334390
:1020B0004E78043136023343019E33600328ECDC52
:1020C0000321A808431C9B002940800003292BD131
:1020D0003849E5185E18A9786D78E35C09042D028B
:1020E000294319433160030008330021FF2B2DDD04
:1020F000314B324919600F21314B196001232749B7
:102100000B60304B19680029FCD006211B680B407E
:10211000042B20D080220020D20593680A318B4303
:102120009360FEBD01217DE7022908D121495D1898
:10213000E1184978E35C090219432960D3E70129D2
:10214000D3D11C495918E35C0B60CCE71948181827
:1021500001600433CAE7002310490B606346002B7B
:102160000CDC3B00FC335A68102101325A6080229B
:10217000D205936801208B439360D2E7009B9B18A4
:102180001B68190A13705170190C1B0ED3700423AD
:102190005B4291709C440432E0E7C046000004407A
:1021A0003C00044038000440340004403000044047
:1021B0000C0004400001044004000440080F00002B
:1021C000100004401400044010B5002901D001F0B3
:1021D000BBFB10BDF7B5604B01919978A1239B0023
:1021E0004B435E4A060014681022E418D6235B00B5
:1021F000E0583623FF33E35C00279343222B41D181
:10220000574B0F3A1A600760012501F0E5FA019B70
:102210001880E8235B00E35C002B01D0B34258DD5B
:102220000023504FFB70AD33FF33E3581A68002A88
:1022300003D09B88DB439B071DD03823FF33E35C2F
:10224000002B18D09B235B00E35C002B13D1D13310
:10225000FF33E35CB3420EDAA4235B00E15AE018DB
:10226000090A023101F048FA23000122FE33013E3F
:1022700001351A87FA70E8235B00E35C002B2AD053
:10228000A8B2FEBD03683D00002BBED0818804309B
:10229000090A023101F030FAD6235B00E3581F60CF
:1022A000B2E72300B133BA00FF3398580137818871
:1022B0000430090A023101F01FFAE8235B00E35CF5
:1022C000BB42EEDCE822F61AED1800235200A354BC
:1022D000A6E70027F1E7200001F00EFB00281FD041
:1022E000002E1DDD7319882647190193B6002000C2
:1022F00001F07AFA5A308000201840680135818850
:102300000430090A023101F0F7F9200001F0A4FAC3
:10231000A3590133A351BD4202D0019B9D42E6D196
:10232000114BE35C002BABD095239B00E35C002BAF
:10233000A6D00E4BE15A0029A2D00D4AA35C9942C7
:1023400002D90133A3549BE700231A212000A35490
:1023500001F0AAFA94E7C046300DFF1F3409FF1FB1
:1023600000140340E010FF1F5A0200007202000038
:102370005E0200000D4970B54A6E0D4CD2038B69A8
:10238000D20BA24206D80B4D0224AA4204D901F076
:1023900083FB70BD02246442E21815007E242540B0
:1023A0002242F4D0A3432B438B61F0E700F00040BE
:1023B0000A200000FC1C00000B001B3B70B5040051
:1023C0003020E02B0DD81300E025493BFF3B9BB2AA
:1023D000ED00AB4205D8034B200019825A8201F070
:1023E000CBF970BD8410FF1FD722044B92009B587D
:1023F00010B5002B00D0984710BDC0460000FF1F4D
:1024000010B501F0B7F8FFF7EFFF2749274BCA6D6A
:10241000274C1A4084235B001343CB65254B1B6874
:10242000186A01F0A1FA244B244A1A60244B254A69
:102430001A60A022244B52001A60244B187801F035
:102440003BF92000224901F0D7FA0023A3600233B0
:10245000A360204B2049236003232048A36001F0A0
:10246000CBFA10221E4BFF201A60802252031A6002
:10247000802292031A60802212041A6001F00CFA82
:10248000012001F089FAFA20400001F0CDFA58202D
:1024900001F042FA134801F027F9012001F0F4F8A5
:1024A000072001F041FA10BD00F0004000FEFEFFE1
:1024B00014100040C45EFF1F000003400180063D71
:1024C000BC00034034080000A40003404A0AFF1F78
:1024D00071020000C3090000FFFF3F002810004008
:1024E00000E100E0307500006B4E336888331B68F4
:1024F00083F3088801F068F9684A69491368002085
:102500000B401360674B684A1B68934200D1ADE0F3
:1025100001F0E2F80221654A13688B431360FFF76C
:102520006FFF634B634C1878C0B201F02DFA0023A3
:10253000A3600233A360604B0120236001F014FA12
:102540000323A36001F058F9040001F00DF9050020
:1025500001F052F9594B186001F0F6F8584B196820
:10256000621A531EA14200D213008022D20393426A
:1025700001D39B029B0A3268D16AC90700D478E074
:1025800050491C0C09689BB24C4359432402090A68
:10259000641803274C49FC3293680A684B489B1A1D
:1025A0004B4A4C4E12684C499B184C4A34609A185E
:1025B0003B400193036892089C46019B0A60634478
:1025C0000360042B03D901323B400A6003600B68AF
:1025D0004349E418200001F077F8424F40493B6836
:1025E000C3183B602000019301F01EF93E4C2068A7
:1025F00008183B492060884205D9019B01333B60A4
:1026000001F012F9216001F0EFF9384B1B78002B33
:102610000ED001F0A9F83168354B4A1B1B6812181F
:102620009A4233D2591A4919091A324801F0E4F989
:10263000314C237A002B0FD001F096F83168E36813
:102640004A1B1218934224D9591A4919091A2B48BE
:1026500001F0D2F900232372294B83F3088801F09B
:10266000D3F9002001F038F801F056F801F034F801
:1026700055E7DC0199000234641A5900641A0921F3
:102680004B438033CB40A408E41882E7FA21890049
:10269000CBE71C49DBE7C046C45EFF1F1CF00040CF
:1026A000FFFFC1FF0C0AFF1FB641210310000040CD
:1026B000490AFF1F14100040C3090000100AFF1F41
:1026C000340AFF1F380AFF1F200AFF1F280AFF1FB6
:1026D0001C0AFF1FB45EFF1F240AFF1FC40900006D
:1026E000710200006008FF1F2C0AFF1F1C09FF1F5A
:1026F000E408FF1F00100040740BFF1F3C10004057
:1027000000000020DC050000A022054B92009B5831
:1027100010B5002B01D0984710BD01F0D5F9FBE7AB
:102720000000FF1FA122054B92009B5810B5002B03
:1027300001D0984710BD01F0C7F9FBE70000FF1F6B
:10274000A222054B92009B5810B5002B01D0984750
:1027500010BD01F0B9F9FBE70000FF1FA322054BF4
:1027600092009B5810B5002B01D0984710BD01F086
:10277000ABF9FBE70000FF1FA422054B92009B581A
:1027800010B5002B01D0984710BD01F09DF9FBE773
:102790000000FF1F70B500F0E7FF4F4B186001F01D
:1027A00073F80400C30702D400F0EEFF70BD0022EE
:1027B0004A4B1A604A4B18780138042829D800F08F
:1027C0004FFF0320181C2400200000F0C5FF012843
:1027D000ECD0444C2378042B6ED100F065FF002828
:1027E000E4D000F0A9FF582001F096F802232370EE
:1027F000DCE7200001F0E0F8E9E7200000F0D4FF7A
:10280000E5E7200000F0C8FFE1E7200001F054F9FF
:10281000DDE701F039F90500012808D1324B1B78BA
:10282000053B012B03D82000FFF76EFFD1E72D4BAE
:102830001B78022B01D0052B20D1022D28D12B4B48
:102840009B7BAB431CD12000FFF76CFF264B187815
:102850000128BED16405BCD4244925224B7B034208
:1028600005D1233A13405A42534126331A000B7DB7
:102870009342AED9322001F0DFF8AAE7022D07D14A
:10288000194B1B78052B11D12000FFF759FFDDE70D
:10289000012D0BD1012B03D12000FFF75FFF98E73B
:1028A000062B03D12000FFF767FF92E7200001F01D
:1028B0000BF9022D8DD1C9E7032B04D10C4B987C69
:1028C00000F0DAFF72E7072B00D06FE7094B987B27
:1028D00000F01AFF6AE7C0469C09FF1F9809FF1F16
:1028E0009009FF1F2309FF1F1C09FF1FA60BFF1FD5
:1028F000BC0BFF1FD40BFF1F10B500F099FE10BDDD
:10290000F7B50B0CFF270122009300233C001E00AB
:102910001D009446019089B262469A40100008401A
:1029200018413618B6B2FF2F02D1012E00D19FB246
:10293000009802401A41AD18ADB2FF2C02D1012D12
:1029400000D19CB20133102BE6D10320012E07D118
:10295000012D04D1019B2401E4191C700138FEBD36
:10296000102EFCD10238102DF9D00230F7E700000C
:102970008023F7B59C46264B264F01932649274ACC
:10298000274D284C284B02281AD160463860086829
:10299000264E30408026360330430860019909787E
:1029A000002909D11660224A2A60224A2260E022C8
:1029B00019689143A03A1BE08021C9021160F2E737
:1029C00066463E600F68194E3E408027FF023E4338
:1029D0000E600199097800290DD1176001280ED1E8
:1029E000154A2A60154A2260E02219689143C03ACC
:1029F0000A431A60F7BD802189021160EEE7E021E9
:102A00000F4A02432A600F4A22601A688A43F0E79D
:102A10004B0AFF1FE0000340D80003409000034032
:102A2000000003405000034040000340FFFFE3FF6D
:102A30000280063D804508220180063D806608220E
:102A40000080069880550822F8B51E4B80261A682B
:102A5000002014003440324232D11A681A4F3243F7
:102A60001A6001223B68063093433B6000F07CFF14
:102A70000122164D2B681E432E603B680A26134325
:102A80003B608027BF00124B1B683B4211D1013EC7
:102A9000F6B2FF2E09D17E220E4B1C682B68E40B88
:102AA0001440934323432B6005E0082000F05CFFB3
:102AB000E9E7002EEFD180222B68600893432B605A
:102AC000F8BDC046C4F000405CF0004018F0004083
:102AD00068F0004060F0004010B500F0CDFF01212B
:102AE0005820034A00F0D8FDFFF7AEFF10BDC046E6
:102AF000600AFF1F10B578220021034800F0A4FFF0
:102B000000F002FF002010BDCC61FF1F70B5040073
:102B100000F0CAFF00230C200B4A010059438D1816
:102B2000515C00290DD0A14208D1012300246B7013
:102B300000F0DAFE00F0D0FF200070BD01330A2B58
:102B4000EBD11224F6E7C046CC61FF1F70B504003C
:102B500000F0AAFF002319001D000D4A107800287C
:102B600006D0A0420CD1557001310C320A29F5D1A2
:102B7000002B0AD100F0C8FE00F0AEFF002070BDAF
:102B80005078461EB0411B18EEE700F0ADFEF3E7AB
:102B9000CC61FF1FF7B504000C20002384460E4DC6
:102BA000019267465F43E85D7E19A04212D000287B
:102BB0000BD10A4B9C4662461B7808331370019B6D
:102BC00070707C557160B360FEBD01330A2BE8D193
:102BD0000320F9E70720F7E7CC61FF1FC861FF1F5B
:102BE0008020F8B5484BC0051B68C1248360474B63
:102BF000FF251A68012313434361454BA4001A685B
:102C0000444B40211A60444B1A68444B1A60444BB1
:102C10001A59AA431A51C52292009E58AE43314315
:102C2000802699509F583F49F6010F403E439E50E1
:102C30009E5880273602360A3043985080201A5911
:102C400000020A4002431A5104341A59364E3F0416
:102C5000324080263A431A511A5936061202120A95
:102C600032431A5108341A5980260A4002431A5135
:102C7000C32292009F58B446AF4337439F509F589A
:102C8000294E0F4007439F509F58374080263604F7
:102C9000374380269F509F5836063F023F0A3743EE
:102CA0009F50C0221F59AF433A431A511A5912027A
:102CB000120A1643C6221E5192009C58AC43654628
:102CC0002C439C509C5800250C4020439850C72012
:102CD00080001A58154C1140C02212020A431A50A3
:102CE000134B1B78DB08AB4201DC0020F8BD2378D6
:102CF000002B06D0A368002B00D0984701350C3478
:102D0000EEE71220F2E7C046E43DFF1FE03DFF1F63
:102D1000B0F00040C461FF1FB4F00040C061FF1F6D
:102D200000E100E0FF00FFFFFFFF00FFCC61FF1F9D
:102D3000C861FF1F030010B51F2809D80722002013
:102D40001340072404490A78A24313430B7010BDB3
:102D500000230620F5E7C046C861FF1F054B064962
:102D60001B780A6805485B0702401B0B13430020D1
:102D70000B607047C861FF1F1CF00040FFFFC1FFE0
:102D800070B50C25FFF7EAFF0A4B1C780A4BE408E4
:102D90006543ED18002C01D1200070BD2B78002B6D
:102DA00006D06B68002B00D09847013C0C3DF1E742
:102DB0001220F2E7C861FF1FC061FF1F1FB500218D
:102DC00002220B0001910091052000F025FE022354
:102DD0000B490A681A42FCD120230393039B5A1E15
:102DE0000392002BFAD1074A1368002BFCDA0B245C
:102DF0006C442000012100F067FD207804B010BD74
:102E000090C8004000C8004013B504000A4B01936D
:102E1000019B002B01D1112016BDFFF7CFFF23002E
:102E20000340044205D0052000F09EFD019B013BBC
:102E3000EDE71800F0E7C046FFFFFF0707B500F019
:102E400033FE80220821D205936A0191002B01D123
:102E50000739916202210C4A11600199481E0190C4
:102E60000029FAD103311160053101910199481E01
:102E700001900029FAD11160002B02D18022D205E5
:102E8000936200F029FE07BD00C00040F0B52D4C54
:102E900089B02378002B4FD1FEF734FD02232A4F4F
:102EA00003903A681A42FCD120230693069B5A1ECF
:102EB0000692002BFAD1254E3368002BFCDA012054
:102EC000FFF7A2FF011E02D0112009B0F0BD0300E0
:102ED00003220190009005AD9F2000F09DFD03218D
:102EE000280000F0F1FC02233A681A42FCD12023AA
:102EF0000793079B5A1E0792002BFAD13368002BC9
:102F0000FCDA0120FFF780FF0028DDD10398FEF7EF
:102F10000DFDAA786B7811041B020B4329780B4333
:102F200063601300113B0A49052B07D80123934026
:102F3000A3600B60012323700020C6E780231B03DE
:102F4000F6E7C046CC3DFF1F90C8004000C80040D7
:102F50009808FF1F1E4B30B55A6818781D4B85B076
:102F6000D31859424B4101210093002300F0F4FC97
:102F7000194B1A4A02259A6300221A6510325A65C3
:102F80008022C4219D65164B1648D202DA6789005B
:102F90004258154B80241A4080231B04134343508E
:102FA000642341200393E40500F006FA402000F07A
:102FB00003FA6562039D6B1E0393002DFAD1032370
:102FC0006362FFF73BFFA562FFF760FF05B030BD0E
:102FD000D83DFF1F95FFFEF700C80040050001FF28
:102FE00004E100E000E100E0FFFF00FFF0B585B084
:102FF0000700FEF787FC022305002D4C22681A42C9
:10300000FCD120230093009B5A1E0092002BFAD182
:10301000284E3368002BFCDA0120FFF7F5FE00286C
:1030200003D01124200005B0F0BD234B2360022300
:1030300022681A42FCD120230193019B5A1E01925F
:10304000002BFAD13368002BFCDA0120FFF7DCFEFD
:103050000028E6D1194B1F60022322681A42FCD1D6
:1030600020230293029B5A1E0292002BFAD133684E
:10307000002BFCDA0120FFF7C7FE0028D1D1104B4E
:103080002360022322681A42FCD120230393039B6E
:103090005A1E0392002BFAD13368002BFCDA012070
:1030A000FFF7B2FE041EBCD12800FEF73FFCB9E7D3
:1030B00090C8004000C8004001000006A8C80040B9
:1030C0000180000110B50020FFF790FF10BD000047
:1030D00010B5064B18705960FFF73CFF0021132014
:1030E000034AFFF757FD002010BDC046D83DFF1F23
:1030F000552FFF1FF0B5040085B003920291FEF733
:1031000001FC882263035B0B52051A438023DB0515
:103110009D6A8023274F0092BA68002601901B0306
:103120009A420CD9F82326001B041E401C4206D0EC
:103130008022214B52025E6219680A431A60002DF8
:103140000BD100F0B1FC02221C4B1A608023DB057E
:103150005A62013A9A6200F0BFFC0023039A93423C
:1031600020D1002D0AD100F09FFC144B03221D60DA
:103170008023DB055A629D6200F0AEFC8023BA68B2
:103180001B039A4208D9002E06D000220A4B0C4994
:103190005A621A680A401A600198FEF7C7FB0020BD
:1031A00005B0F0BD009A0299D2181278CA540133C2
:1031B000D4E7C046CC3DFF1F00C8004000C000401F
:1031C000FFFFFEFFF0B587B0029103920400FEF707
:1031D00099FB019000F068FC802302250122234E18
:1031E000DB0535605D629A6200F076FC204F3B683B
:1031F0002B42FCD120230493049B5A1E0492002BE3
:10320000FAD11C4D2B68002BFCDA0120FFF7FCFDE6
:10321000002802D0112007B0F0BD2000039A0299C7
:1032200000F0CAFA022304003A681A42FCD12023B3
:103230000593059B5A1E0592002BFAD12B68002B93
:10324000FCDA0120FFF7E0FD051EE3D100F02CFCC5
:1032500080230322DB0535605A629D6200F03CFC4E
:103260000198FEF763FBE0B2D5E7C04600C000401E
:1032700090C8004000C80040F0B5802489B0060026
:10328000FEF740FBE405A36A02250393029000F0D9
:103290000BFC0123304F3D606562A36200F01CFC13
:1032A0002E4C23682B42FCD120230593059B5A1EEC
:1032B0000592002BFAD12A4D2B68002BFCDA012055
:1032C000FFF7A2FD002803D01124200009B0F0BDB3
:1032D000244B2360022322681A42FCD12023069348
:1032E000069B5A1E0692002BFAD12B68002BFCDAA3
:1032F0000120FFF789FD021EE6D11B4B03211E6052
:10330000030001900090202000F086FB0223226839
:103310001A42FCD120230793079B5A1E0792002BC9
:10332000FAD12B68002BFCDA0320FFF76DFD041E99
:10333000CAD100F0B9FB80230322DB053C605A624E
:103340009C6200F0C9FB039B002B01D1FFF776FDC7
:103350000298FEF7EBFAB8E700C0004090C80040C2
:1033600000C800400100000694C8004007B50002F4
:1033700001910422000A01A9FFF724FF0EBD0000FD
:1033800073B5050005240B4AA3005B429B1819681E
:103390006B46DE1D3000FFF7B3FA022804D1337804
:1033A0002B55013CEFD276BD052CFCD00128FAD17B
:1033B0000230F8E7140900111F2807D801238022E2
:1033C0008340D20591680B43936070473F2808D82B
:1033D0000123802220388340D20551690B43536179
:1033E000F3E75F28F1D80123802240388340D205DB
:1033F000116A0B431362E8E71F2807D801228021D6
:103400008240C9058B6893438B6070473F2808D87A
:103410000122802120388240C9054B6993434B61CA
:10342000F3E75F28F1D80122802140388240C905A6
:103430000B6A93430B62E8E71F2810D88023020031
:10344000DB05153A1968012A06D820229143196034
:1034500019680A431A60704701228240F6E73F2844
:1034600011D880230200DB05353AD968032A06D833
:1034700010229143D960D9680A43DA60EBE7012250
:1034800020388240F5E75F28E5D842238022181AC9
:10349000413B8340D205516A99435162516A0B43C3
:1034A0005362D8E710B50400012813D1A0221849AF
:1034B00092050B685B015B0913430B60154B164AC1
:1034C00019681140154A0A431A60402219680A43D4
:1034D0001A6010BD0028FCD101000A2000F094F908
:1034E00021000B2000F090F9C0220A4B92001968CD
:1034F0000A4340211A601A688A431A60B0220449BC
:1035000012060B685B015B0913430B60E1E7C046E1
:1035100014F000401CF000407F00FEFF80FD010021
:1035200072B6074A1368013313600422054B1A6010
:103530000023054A13608022D2055360FEE7C0468F
:103540007808FF1FC0F00040C4F0004005490B6838
:10355000002B05D1044A0A6004490A60044A13603A
:103560007047C046140AFF1F841E0000380AFF1F60
:10357000C4F000400023034A1360034A1360034A67
:103580001360704754F0004040F1004044F10040A7
:10359000002310B5184C8AB0009301932378012BB7
:1035A00027D06946012000F097F9002817D1009B29
:1035B00012490293019B06AA0393114B02A81B68B0
:1035C0000493104B1B68059300F0B6F910220E49C6
:1035D00006A800F049FA002804D1FF232370002038
:1035E0000AB010BD0123094A074902A8237000F060
:1035F000A3F90120F4E7C046C85EFF1F102900119F
:10360000082900110C29001120290011CC5EFF1F90
:1036100013B501246946012000F05EF9034B0094C4
:103620000193FFF7B5FF200016BDC046BB0B00009D
:1036300010B5FFF79FFFFFF7EBFF002802D0024B0A
:10364000984710BDFEE7C046E1A2000002B47146F3
:1036500049084900095649008E4402BC7047C046DB
:1036600002B4714649084900095C49008E4402BC15
:103670007047C04603B47146490840004900095AE2
:1036800049008E4403BC704701B40248844601BC23
:10369000604700BFE512010001B40248844601BC46
:1036A000604700BF0167010001B40248844601BCC5
:1036B000604700BF01D7000001B40248844601BC46
:1036C000604700BFEDA5000001B40248844601BC7C
:1036D000604700BF090E000001B40248844601BCE7
:1036E000604700BF016C010001B40248844601BC80
:1036F000604700BF8D11010001B40248844601BC3F
:10370000604700BFC115010001B40248844601BCF6
:10371000604700BFC1F7000001B40248844601BC05
:10372000604700BF8552010001B40248844601BCD5
:10373000604700BF8D82000001B40248844601BC8E
:10374000604700BF6DF6000001B40248844601BC2A
:10375000604700BFC166010001B40248844601BC55
:10376000604700BF0134010001B40248844601BC37
:10377000604700BFC95C010001B40248844601BC37
:10378000604700BF116E000001B40248844601BCCE
:10379000604700BFDD0A010001B40248844601BC55
:1037A000604700BFF535010001B40248844601BC02
:1037B000604700BF0534010001B40248844601BCE3
:1037C000604700BF9573010001B40248844601BC04
:1037D000604700BFC9A9000001B40248844601BC8B
:1037E000604700BFCD0C010001B40248844601BC13
:1037F000604700BFD9B0000001B40248844601BC54
:10380000604700BF156B010001B40248844601BC4B
:10381000604700BFBDA1001101B40248844601BC4D
:10382000604700BF2144000001B40248844601BC47
:10383000604700BF090E000001B40248844601BC85
:10384000604700BFBD5C010001B40248844601BC72
:10385000604700BF51B8000001B40248844601BC73
:10386000604700BF5976010001B40248844601BC9C
:10387000604700BF85C1000001B40248844601BC16
:10388000604700BF4DF9000001B40248844601BC06
:10389000604700BFBD0B010001B40248844601BC73
:1038A000604700BFED6B010001B40248844601BCD3
:1038B000604700BF53B9000001B40248844601BC10
:1038C000604700BF15B5001101B40248844601BC31
:1038D000604700BF3D71010001B40248844601BC4D
:1038E000604700BFE1AC000001B40248844601BC5F
:1038F000604700BF21A9000001B40248844601BC12
:10390000604700BF71B0000001B40248844601BCAA
:10391000604700BFADAE000001B40248844601BC60
:10392000604700BF7912010001B40248844601BC1F
:10393000604700BFF90D010001B40248844601BC94
:10394000604700BFDD3F000001B40248844601BC6F
:10395000604700BFE9D4000001B40248844601BCBE
:10396000604700BFC56D010001B40248844601BC38
:10397000604700BF0189000001B40248844601BCD1
:10398000604700BFE94C010001B40248844601BC15
:10399000604700BF8914010001B40248844601BC9D
:1039A000604700BF6911010001B40248844601BCB0
:1039B000604700BFE927000001B40248844601BC0B
:1039C000604700BF0934010001B40248844601BCCD
:1039D000604700BFE90B010001B40248844601BC06
:1039E000604700BF6D0B010001B40248844601BC72
:1039F000604700BFD544010001B40248844601BCC1
:103A0000604700BF2D6C010001B40248844601BC30
:103A1000604700BF7997000001B40248844601BCAA
:103A2000604700BF496D010001B40248844601BCF3
:103A3000604700BF8512010001B40248844601BC02
:103A4000604700BF6137010001B40248844601BCF1
:103A5000604700BFB70E000001B40248844601BCB5
:103A6000604700BF8944000001B40248844601BC9D
:103A7000604700BFCD4C010001B40248844601BC40
:103A8000604700BFED68010001B40248844601BCF4
:103A9000604700BFDD0C010001B40248844601BC50
:103AA000604700BFD1AE000001B40248844601BCAB
:103AB000604700BF75A9000001B40248844601BCFC
:103AC000604700BFF935010001B40248844601BCDB
:103AD000604700BFE917010001B40248844601BCF9
:083AE000604700BF9DA9000032
:103AE80002000000AABD001101000000BCBB0011CB
:103AF80002000000A6BD001101000000283BFF1FC6
:103B080002000000C4BB001101000000385CFF1F68
:103B180002000000A4BD001103000000AC5BFF1F01
:103B28001200000002000000AABD00110100000000
:103B380004BC001102000000A6BD00110100000035
:103B480001BC0011020000000EBC001103000000BF
:103B5800E75BFF1F02000000A4BD00110300000086
:103B6800FC5BFF1F02000000A6BD00110100000061
:103B780000BC0011020000000CBC00110300000092
:103B8800BD5BFF1F02000000A4BD00110300000080
:103B9800DE5BFF1F02000000AABD0011010000004B
:103BA80044BC001102000000A6BD00110100000085
:103BB800713CFF1F0200000056BC0011010000000C
:103BC8003FBC001102000000A6BD0011010000006A
:103BD800703CFF1F0200000054BC001101000000EF
:103BE800045CFF1F02000000A6BD001101000000D8
:103BF8006F3CFF1F0200000052BC001101000000D2
:103C08002FBC001102000000A6BD00110100000039
:103C18006E3CFF1F0200000050BC001101000000B4
:103C28002ABC001102000000A6BD0011010000001E
:103C38006D3CFF1F020000004EBC00110100000097
:103C480025BC001102000000A6BD00110100000003
:103C58006C3CFF1F020000004CBC0011010000007A
:103C680020BC001102020202020200000000000053
:103C78000D0C0000654B00112B4B001198BC001176
:103C880090011D0018001800FFFF0701020304053A
:103C9800060201060000000000000000000000000D
:103CA800000000000000000000000000000000000C
:103CB8000300000002000000AABD0011010000007E
:103CC800B8BC001102000000A6BD001101000000F0
:103CD8002C3DFF1F02000000C2BC001101000000C3
:103CE800325CFF1F02000000A4BD001103000000A9
:103CF8009C5EFF1F02000000A6BD0011010000002D
:103D08002C3DFF1F02000000C0BC00110100000094
:103D1800345CFF1F02000000A4BD00110300000076
:103D2800945EFF1F126C6C6C00000000005800408D
:103D3800151600000001000000000111FFFF00003F
:103D48005048593600000000000000000B00050034
:103D5800F0000000B4000028002800283075A000FA
:103D6800A000A000A00000080008E001F00010007A
:103D780010001000100010001000500050005000FB
:103D880010001000D0070000000000000F00010024
:103D98000500307507001000010081FF00000000D9
:103DA800FF000000A5730011AD7100113D6F0011F7
:103DB800FFFF0100FF000000C19D00113D9B0011A5
:103DC800559A0011000000000000000000000800E3
:103DD800040000003B0001085902E0018821280086
:103DE80002000000AABD00110100000070BE001111
:103DF80002000000A6BD001101000000653EFF1F83
:103E080002000000A2BD0011010000008462FF1F33
:103E180002000000A6BD001101000000643EFF1F63
:103E280002000000A0BD001101000000623EFF1F5B
:103E380002000000A6BD001101000000603EFF1F47
:103E4800020000009EBD001101000000583EFF1F47
:103E5800180018001D009001020000030202000073
:103E680002000000AABD00110100000084BE00117C
:103E780002000000A6BD001101000000A83EFF1FBF
:103E8800020000009CBD00110000000000000000BE
:103E980002000000A4BD001103000000A462FF1F7F
:023EA80020FFF9
:040000051FFF184180
:00000001FF
